:020000040000FA
:200000000C943F0F0C9408120C94520F0C94520F0C94520F0C94520F0C94520F0C943A1544
:200020000C94520F0C94520F0C94520F0C941C130C94520F0C94520F0C94A7120C94520F92
:200040000C94520F0C94520F0C9447140C94520F0C9420140C94520F0C94520F0C94520FCB
:200060000C94520F0C94520F4000005600014000012A00010A0000040000080201810000E1
:200080005600004A616E1F4665621C4D61721F4170721E4D61791F4A756E1E4A756C1F410D
:2000A00075671F5365701E4F63741F4E6F761E4465631F53756E646179004D6F6E64617962
:2000C0000054756573646179005765646E65736461790054687572736461790046726964C4
:2000E000617900536174757264617900B300BA00C100C900D300DC00E3000003030601043F
:20010000060205000305205465726D696E616C00808386898C8F9295989C9FA2A5A8ABAEFF
:20012000B0B3B6B9BCBFC1C4C7C9CCCED1D3D5D8DADCDEE0E2E4E6E8EAECEDEFF0F2F3F5EE
:20014000F6F7F8F9FAFBFCFCFDFEFEFFFFFFFFFFFFFFFFFFFFFFFEFEFDFCFCFBFAF9F8F718
:20016000F6F5F3F2F0EFEDECEAE8E6E4E2E0DEDCDAD8D5D3D1CECCC9C7C4C1BFBCB9B6B368
:20018000B0AEABA8A5A29F9C9895928F8C898683807C797673706D6A6763605D5A5754513E
:2001A0004F4C494643403E3B383633312E2C2A272523211F1D1B1917151312100F0D0C0A30
:2001C0000908070605040303020101000000000000000000000001010203030405060708C6
:2001E000090A0C0D0F1012131517191B1D1F212325272A2C2E313336383B3E404346494C36
:200200004F5154575A5D6063676A6D707376797C4A645200010204081020408042005000FC
:200220004700303132333435363738394142434445460CF80C46F846F8F80CF8FF01FE014E
:2002400001FE01FEFE01FEFE010101FEFE01FE0101FE01FEFEFF0B694F0B8C4FFF0B697F10
:200260000B8C4FFF0B694F0B8C7FFF56025D0264020B694F0B8C4F0BAF4FFF0B697F0B8C69
:200280004F0BAF4FFF0B694F0B8C7F0BAF4FFF0B697F0B8C7F0BAF4FFF0B694F0B8C4F0B61
:2002A000AF7FFF0B697F0B8C4F0BAF7FFF71027B0285028F029902A3020B694F0B8C4F0B04
:2002C000AF4F0BD24FFF0B697F0B8C4F0BAF4F0BD24FFF0B694F0B8C7F0BAF4F0BD24FFFDB
:2002E0000B697F0B8C7F0BAF4F0BD24FFF0B694F0B8C4F0BAF7F0BD24FFF0B697F0B8C4FDB
:200300000BAF7F0BD24FFF0B694F0B8C7F0BAF7F0BD24FFF0B697F0B8C7F0BAF7F0BD24FCE
:20032000FF0B694F0B8C4F0BAF4F0BD27FFF0B697F0B8C4F0BAF4F0BD27FFFB902C602D31E
:2003400002E002ED02FA020703140321032E030C0102030405060708090A0B0C01020304F4
:2003600005060708090A0B0000010001010001FF01FF00FFFF00FF53657269616C20496E0E
:20038000204F766572666C6F77200A0D004E6F726D616C0053686F72742053312020204DE8
:2003A000656E75004C6F6E67202053312020204368616E67650053686F7274205332202006
:2003C0002048656C70004C6F6E67202053322020205265626F6F74004368616E67652F4D92
:2003E000656E75005331202020202020202020496E6372656D656E74005332202020202047
:2004000020202020416476616E636500526566726573683A00557054696D653A00F1061903
:20042000EBFD06A9EB8D0355CD94030AB8A4030AA3B6030A8EC6030A79D8033C5FE4030AD7
:200440004AF9030A350C040A1915040A0400008E1900008E04434D564B00FC23EF240524F8
:20046000AA2577077D07740786074E464A50554C4200B425A7279E27B827FA24DC24F22314
:200480000505040302030944544148494F52535747000C2D532DBD2D962BC32C7F2BB42B65
:2004A000BA2BEB2B6E2F20415652204F7363696C6C6F73636F706520436C6F636B2000312F
:2004C0002064696769742076616C75652028302D003220646967697420006872733A2000DF
:2004E0006D696E733A2000736563733A2000796561723A20006D6F6E74683A20006461791A
:200500003A200043616E63656C2F54696D656F7574004E616D65200028432932303231200B
:200520004A616E20646520526965000D0A00342068657820646967697420494F43544C3AC3
:2005400020004453542066697820002048656C703A0D0A413A204170706C69636174696F6E
:200560006E2053656C656374696F6E2028302E2E35290D0A423A204275726E2D696E207037
:20058000726576656E74696F6E0D0A433A20416C61726D206F6E2F6F66660D0A443A204381
:2005A00068616E676520446174650D0A463A20436C6F636B2046616365204D6F646520287B
:2005C000302E2E35290D0A473A2047505320496E7075740D0A483A2048656C700D0A493A83
:2005E00020494F43544C0D0A4A3A204E616D65204D6F64652028302E2E34290D0A4B3A2092
:200600004368726F6E6F20446973706C61790D0A4C3A204C454420626C696E6B696E670D6E
:200620000A4D3A205050532054726967676572204D6F64650D0A4E3A204E756D65726963EB
:2006400020446973706C6179204D6F64652028302E2E35290D0A503A20506C6179204D6F9A
:2006600064652028302E2E33290D0A523A20526573657420454550726F6D20436F6E666964
:20068000670D0A533A20446973706C6179205374617475730D0A543A204368616E6765208A
:2006A00054696D650D0A553A204368616E676520445354206D6F64650D0A563A20566572DB
:2006C000626F7365204F75747075740D0A573A204368616E6765204E616D6500436F6D6D85
:2006E000616E64284820666F722068656C70293A00447574636874726F6E69780056342E70
:20070000330001010101010001010101000001010100000001010000000001000000000097
:20072000010000000001010000000101010000010101010080FE80F2008DFE8CF9009AFC19
:2007400099F700A6F8A5F400B3F4B1EF00BFEEBAE500CAE6C7E200D4DED0DA00DDD5D9D12E
:2007600000E5CBE1C800EDBFE4BA00F3B4EEB200F7A7F3A600FB9BF69A00FD8EF88D00FD25
:2007800080F18000FD73F87400FB66F66700F75AF35B00F34DEE4F00ED41E44600E536E15E
:2007A0003900DD2CD93000D423D02700CA1BC71F00BF13BA1C00B30DB11200A609A50D00A9
:2007C0009A05990A008D038C08007F037F0F0072037308006505660A0059095A0D004C0DB7
:2007E0004E12004113461C00351B381F002B232F2700222C2630001A361E390012421B4797
:20080000000C4D114F00085A0C5B000466096700027307740002810E8100028E078D000452
:200820009B099A0008A70CA6000CB411B20012BF1BBA001ACB1EC80022D526D1002BDE2FFF
:20084000DA0035E638E20040EE45E5004CF44EEF0059F85AF40065FC66F70072FE73F9FF7C
:2008600080FE80FD81FD81FC008DFE8DFD8EFD8EFC009AFC99FB9BFB9AFA00A6F8A6F7A722
:20088000F7A7F600B3F4B2F3B4F3B3F200BFEEBEEDC0EDBFEC00CAE6C9E6CBE5CAE500D4EA
:2008A000DED3DDD5DDD4DC00DDD5DCD4DED4DDD300E5CBE5CAE6CAE6C900EDBFECBFEEBEC3
:2008C000EDBE00F3B4F2B3F4B3F3B200F7A7F6A7F8A6F7A600FB9BFA9AFC9AFB9900FD8E80
:2008E000FC8EFE8DFD8D00FD80FC80FE81FD8100FD73FC73FE74FD7400FB66FA67FC67FB81
:200900006800F75AF65AF85BF75B00F34DF24EF44EF34F00ED41EC42EE42ED4300E536E569
:2009200037E637E63800DD2CDC2DDE2DDD2E00D423D324D524D42500CA1BC91BCB1CCA1CA7
:2009400000BF13BE14C014BF1500B30DB20EB40EB30F00A609A60AA70AA70B009A05990647
:200960009B069A07008D038D048E048E05007F037F04800480050072037204730473050007
:200980006505660666066707005909590A5A0A5A0B004C0D4D0E4D0E4E0F004113411442C2
:2009A00014421500351B361B361C371C002B232C242C242D2500222C232D232D242E001AEC
:2009C000361A371B371B38001242134213431443000C4D0D4E0D4E0E4F00085A095A095B00
:2009E0000A5B00046605670567066800027303730374047400028103810382048200028E66
:200A0000038E038D048D00049B059A059A06990008A709A709A60AA6000CB40DB30DB30E9C
:200A2000B20012BF13BF13BE14BE001ACB1ACA1BCA1BC90022D523D423D424D3002BDE2C1B
:200A4000DD2CDD2DDC0035E636E636E537E50040EE41ED41ED42EC004CF44DF34DF34EF281
:200A60000059F859F75AF75AF60065FC66FB66FB67FA0072FE72FD73FD73FCFF7AEB7AD93B
:200A80000080E883EB89EB8CE88CE580D98CD900B5E4B5D20000D2BBD5BEDBBEDEBBDEB861
:200AA000D2ACDEAC0000E286E589EB89EE86EE83EB80EE7DEE7AEB77E577E27A00E580EB57
:200AC0008000E04CD44CDD55DD430000B831AC31AC28B528B825B822B51FAF1FAC2200005A
:200AE000852182247C24792179157C12821285158518821B7C1B79180047315331532E50F7
:200B00002B4D254D1F00224C1F4F1F52225528552B522B4F284C224C1F491F462243284315
:200B20002B462B49284C00001D841A811A81148111841187148A1A8A1D871D7B1A78147827
:200B4000117B000021BE21AC000027BB2ABE30BE33BB33AF30AC2AAC27AF27BB000049E43E
:200B600049D2000053E453D2FF0073EF76F27CF27FEF7FEC73E07FE0008DE981E98AF28A56
:200B8000E000AAE2AAD00000B0DFB3E2B9E2BCDFBCDCB9D9BCD6BCD3B9D0B3D0B0D300B388
:200BA000D9B9D900D0BCD0AA0000E2B3D6B3DFBCDFAA0000DC89DC7700EE89E289E280EB9B
:200BC00080EE7DEE7AEB77E577E27A00D055D0430000E252DF55D955D652D646D943DF4358
:200BE000E246E249DF4CD94CD6490000AA2DAA1B0000B02DBC2DBC2AB927B621B61B000063
:200C00007B217B0F008318801B801E832189218C1E8C1B8918831880158012830F890F8C22
:200C2000128C15891800492F491D00005B295826582652264F294F2C522F582F5B2C5B208D
:200C4000581D521D4F2000001E52215527552A522A4F1E432A4300002F52325538553B52FA
:200C60003B46384332432F462F5200001187148A1A8A1D871D8411781D780000238A237888
:200C800000001EBB21BE27BE2ABB2AB81EAC2AAC00002FBB32BE38BE3BBB3BB82FAC3BACD5
:200CA000000040DD43E049E04CDD4CDA40CE4CCE000051DD54E05AE05DDD5DDA5AD75DD4E5
:200CC0005DD15ACE54CE51D10054D75AD7FF76DF8ADF0079DF80F30079F380DF0083DF83E6
:200CE000F30087F387DF0076F38AF300ADD1B5D100B1D1B1E500ADE5B5E50000D2ABDEABED
:200D000000D6ABD6BF00DAABDABF00D2BFDEBF00DC76EE7600E076E08A00E576E58A00EA47
:200D200076EA8A00DC8AEE8A00C942DF4200CE42CE5600D242D25600D642D65600DA42DA15
:200D40005600C956DF560000A922B92200AD36B122B53600A936B936000075148914007935
:200D6000287D1481280085148528007528892800432259220046364A224E36005122513637
:200D80000055225536004336593600001D42394200225626422A56002E422E560032423275
:200DA000560036423656001D5639560011772377001477148B001877208B00188B20770017
:200DC000118B238B000024AB32AB0027AB2FBF0027BF2FAB0024BF32BF0048D15AD1004B3A
:200DE000D153E5004BE553D10056D156E50048E55AE5FF007AEB7AD90080E883EB89EB8C3B
:200E0000E88CE580D98CD900E286E589EB89EE86EE83EB80EE7DEE7AEB77E577E27A00E54F
:200E200080EB8000852182247C24792179157C12821285158518821B7C1B7918001D841ADA
:200E4000811A81148111841187148A1A8A1D871D7B1A781478117BFF80EC8080FF8BEC802B
:200E600080FF96EA8080FFA1E78080FFABE38080FFB6DE8080FFBFD88080FFC8D18080FF9F
:200E8000D0C98080FFD7C08080FFDDB68080FFE2AC8080FFE6A28080FFE9978080FFEB8C88
:200EA0008080FFEB808080FFEB758080FFE96A8080FFE65F8080FFE2558080FFDD4A808077
:200EC000FFD7418080FFD0388080FFC8308080FFBF298080FFB6238080FFAB1E8080FFA1D6
:200EE0001A8080FF96178080FF8B158080FF80158080FF74158080FF69178080FF5E1A80FB
:200F000080FF541E8080FF4A238080FF40298080FF37308080FF2F388080FF28418080FFD9
:200F2000224B8080FF1D558080FF195F8080FF166A8080FF14758080FF14808080FF148C23
:200F40008080FF16978080FF19A28080FF1DAC8080FF22B68080FF28C08080FF2FC98080AE
:200F6000FF37D18080FF40D88080FF49DE8080FF54E38080FF5EE78080FF69EA8080FF74EE
:200F8000EC8080FF828080E67E808280FF81808AE67E818180FF818095E47E818180FF8195
:200FA000809FE27E818180FF8180A9DE7E818180FF817FB3D97E82817FFF817FBBD37E8291
:200FC000817FFF817FC4CC7E82817FFF817FCBC57E82817FFF817FD2BC7E82817FFF807F68
:200FE000D8B37F82807FFF807FDDAA7F82807FFF807FE1A07F82807FFF807FE3967F82806A
:201000007FFF807FE58B7F82807FFF7F7EE58080827F7EFF7F7FE57680827F7FFF7F7FE34B
:201020006B80827F7FFF7F7FE16180827F7FFF7F7FDD5780827F7FFF7E7FD84D81827E7FB4
:20104000FF7E7FD24581827E7FFF7E7FCB3C81827E7FFF7E7FC43581827E7FFF7E7FBB2EA0
:2010600081827E7FFF7E7FB32881827E7FFF7E80A92381817E80FF7E809F1F81817E80FF16
:201080007E80951D81817E80FF7E808A1B81817E80FF7E817F1B82807E81FF7E81751B8156
:2010A000807E81FF7E816A1D81807E81FF7E81601F81807E81FF7E81562381807E81FF7EBB
:2010C000814D2881807E81FF7E82442E817F7E82FF7E823B35817F7E82FF7E82343C817FCB
:2010E0007E82FF7E822D45817F7E82FF7F82274E807F7F82FF7F822257807F7F82FF7F8291
:201100001E61807F7F82FF7F821C6B807F7F82FF7F821A76807F7F82FF80821A817F7E8020
:2011200082FF80821A8B7F7F8082FF80821C967F7F8082FF80821EA07F7F8082FF808222F2
:20114000AA7F7F8082FF808227B37F7F8082FF81822DBC7E7F8182FF818234C57E7F818224
:20116000FF81823BCC7E7F8182FF818244D37E7F8182FF81824CD97E7F8182FF818156DEF1
:201180007E808181FF818160E27E808181FF81816AE47E808181FF818175E67E808181FF62
:2011A000828080BC7E808280FF818086BC7E818180FF81808CBB7E818180FF818092BA7E9E
:2011C000818180FF818098B77E818180FF817F9EB47E82817FFF817FA3B17E82817FFF811A
:2011E0007FA8AD7E82817FFF817FACA97E82817FFF817FB0A47E82817FFF807FB39E7F8224
:20120000807FFF807FB6997F82807FFF807FB9937F82807FFF807FBA8D7F82807FFF807FF5
:20122000BB877F82807FFF7F7EBB8080827F7EFF7F7FBB7A80827F7FFF7F7FBA7480827F58
:201240007FFF7F7FB96E80827F7FFF7F7FB66880827F7FFF7E7FB36281827E7FFF7E7FB013
:201260005D81827E7FFF7E7FAC5881827E7FFF7E7FA85481827E7FFF7E7FA35081827E7F2A
:20128000FF7E7F9E4D81827E7FFF7E80984A81817E80FF7E80924781817E80FF7E808C46E3
:2012A00081817E80FF7E80864581817E80FF7E817F4582807E81FF7E81794581807E81FFE8
:2012C0007E81734681807E81FF7E816D4781807E81FF7E81674A81807E81FF7E81624D81C7
:2012E000807E81FF7E825C50817F7E82FF7E825754817F7E82FF7E825358817F7E82FF7EF3
:20130000824F5D817F7E82FF7F824C63807F7F82FF7F824968807F7F82FF7F82466E807F8C
:201320007F82FF7F824574807F7F82FF7F82447A807F7F82FF808244817F7E8082FF80826F
:2013400044877F7F8082FF8082458D7F7F8082FF808246937F7F8082FF808249997F7F80B4
:2013600082FF80824C9E7F7F8082FF81824FA47E7F8182FF818253A97E7F8182FF818257B4
:20138000AD7E7F8182FF81825CB17E7F8182FF818261B47E7F8182FF818167B77E8081815B
:2013A000FF81816DBA7E808181FF818173BB7E808181FF818179BC7E808181FF059419945B
:2013C000196C056C059406951A951A6D066D0695FF0F6C0F941094106CFF05941994198084
:2013E0000580056C196C1A6D066D067F1A7F1A930693FF05941994196C056C066D1A6D1AC5
:2014000095069500058018800018810681FF0594058018800018810681069500196C1994BD
:201420001A951A6DFF1994059405801980196D066D056C196C001A6D1A81068106951A9531
:20144000FF0594056C196C198006800006811A811A6D066D0695FF05941994196C1A6D1ABD
:20146000950695FF05941994196C056C059406951A951A6D066D06950006801880001881D2
:201480000681FF056C196C1994059405801880001881068106951A951A6D066DFFBC13D16A
:2014A00013DA13F3130E1425144114571464148314058406840685058500057C067C067B50
:2014C000057B004C844D844D854C85004C7C4D7C4D7B4C7BFF10383810100010006C6C4859
:2014E000000000000000287C28287C2800203840300870100064640810204C4C00205050AC
:201500002054483400303020000000000010202020202010002010101010102000002838AB
:201520007C382800000010107C10100000000000000060604000000078000000000000009B
:201540000000303000000408102040000038444C546444380010301010101038003844047B
:201560001820407C003844043804443800081828487C0808007C40407804443800182040B7
:2015800078444438007C0408102020200038444438444438003844443C04083000000060CB
:2015A00060006060000000303000303020081020402010080000007C00007C00002010084B
:2015C0000408102000384404181000100038445C545C403800384444447C4444007844440F
:2015E0007844447800384440404044380078444444444478007C40407840407C007C40400B
:2016000078404040003844405C44443C004444447C444444003810101010103800040404D6
:20162000044444380044485060504844004040404040407C00446C544444444400446454C2
:201640004C44444400384444444444380078444478404040003844444454483400784444A2
:20166000784844440038444038044438007C10101010101000444444444444380044444436
:20168000444428100044445454545428004444281028444400444444281010100078081066
:2016A000204040780038202020202038000040201008040000380808080808380010284472
:2016C000000000000000000000000000FC3030100000000000000038043C443C00404078AE
:2016E0004444447800000038444044380004043C4444443C0000003844784038001820205E
:20170000782020200000003C44443C0438404070484848480010001010101018000800181D
:20172000080808483040404850605048001010101010101800000068545444440000007089
:2017400048484848000000384444443800000078444444784000003C4444443C0400005891
:201760002420207000000038403804380000207820202810000000484848582800000044FD
:20178000444428100000004444547C280000004848304848000000484848381060000078C1
:2017A0000830407800182020602020180010101000101010003008080C08083000285000C5
:2017C0000000000000387C7C7C7C7C3800596F7572204E616D6520686572650042696E619F
:2017E000727920436C6F636B004469676974616C20436C6F636B00506C6179204D6F6465ED
:20180000004C45442054696D65005761726E696E6773004F6E2053637265656E204D656E7E
:2018200075005468616E6B20596F750042692D48657820436C6F636B00446179206F6620A4
:20184000746865205765656B0043616C6962726174696F6E2053637265656E005465726D1B
:20186000696E616C0053636F72653A2020323333303000566563746F722047726170686968
:2018800063730048656C702053637265656E004275726E496E2050726576656E74696F6ED1
:2018A00000416C736F20537570706F7274656400475053204E4D45412050617273696E6794
:2018C000004461796C6967687420536176696E672054696D6500416C61726D0033372043E1
:2018E0006F6D62696E6174696F6E7300546869732064656D6F206D6F64652073686F7773CF
:2019000020736F6D65206F6620746865206361706162696C6974696573206F66207468653D
:201920000D0A41565220436C6F636B2E205468652064656D6F207072657365727665732048
:20194000746865207374617465206F6620796F757220636C6F636B0D0A00000000FF00FFE0
:20196000FFFFFFFFFF00FF0000005E6A695D695D6F676F675E6A695D80508050875B875B7B
:201980006F6780508548875B905A7C02830783078B028B02860986098B118B11830C830CE8
:2019A0007C117C11810981097C0284528B578B57935293528E598E59936193618B5C8B5C93
:2019C0008461846189598959845272C079C579C581C081C07CC77CC781CF81CF79CA79CAC7
:2019E00072CF72CF77C777C772C016F419F619F61DF41DF41AF71AF71DFB1DFB19F819F8F9
:201A000016FB16FB18F718F716F4871E8E238E23961E961E91259125962D962D8E288E28AF
:201A2000872D872D8C258C25871E3E8A438D438D498A498A448F448F499549954390439021
:201A40003E953E95418F418F3E8AA2A8A9ADA9ADB1A8B1A8ACAFACAFB1B7B1B7A9B2A9B294
:201A6000A2B7A2B7A7AFA7AFA2A866DC6DE16DE175DC75DC70E370E375EB75EB6DE66DE632
:201A800066EB66EB6BE36BE366DC1A38213D213D29382938243F243F29472947214221428A
:201AA0001A471A471F3F1F3F1A38A86EAF73AF73B76EB76EB275B275B77DB77DAF78AF78AE
:201AC000A87DA87DAD75AD75A86E468647874A824B834E7E4F7F2DD82ED94875497630D20A
:201AE00031D333CC34CD26A627A76069616A41707000436C6F636B0043616C005465726DFF
:201B00000047656E00426F6F740044656D6F00505053004E756D004C6564004275726E695A
:201B20006E004469616C004F6E004F666600313268720032346872004865780044617465C5
:201B400000416C61726D004469670042696E00526F6D004D696E004D6F7273650044656208
:201B6000756700506C6179004E6F726D00526576004646004652004E616D650045646974FF
:201B8000004461790044656274005075736820533120746F20537461727400475053004FFA
:201BA0006666002D3132002D3131002D3130002D3920002D3820002D3720002D3620002D6D
:201BC0003520002D3420002D3320002D3220002D312000302020002B3120002B3220002B1E
:201BE0003320002B3420002B3520002B3620002B3720002B3820002B3920002B3130002BD2
:201C00003131002B313200445354004368726F6E6F0052657365740031487A0034303936B7
:201C2000487A00426175640031393230302000323838303020003338343030200035373667
:201C4000303020003131353230300032353030303000343830302020003936303020200099
:201C60003134343030200055534100455500350036003700380039003000310032003300EF
:201C800034002E1B331B4F1B471B4B1B531B2E1B331B381B3C1B411B2A1B271B571B5D1BCB
:201CA0002A1B281C2F1C361C3D1C441C4B1C521C591C601C2A1B271B181C1C1CC31BC71BCC
:201CC000CB1BCF1BD71BDB1BDF1BE31B007FFCFDFEFF0102030402030405FF0607080900AA
:201CE000681B6D1B711B741B271B2A1B7C1B811B851B671C6B1C2A1BF21AF81AFC1A011BC5
:201D00000A1B051B6034CC365B060634C1366306C63249366B0670338A367306003335328F
:201D20007B06E3325036830638336D368B06EB33B6369306C933AB369B06A733A036A306E5
:201D40008D339536AB061D336236B30653337836BB06AA322A36BF06783284340000292AFB
:201D6000463601802A2B523202802B2C5B3203802CB1613200002D2EB031DC042E2F523237
:201D8000D4042F305B32CC0430B1613200003475B231DC0435765232D40436775B32CC04BE
:201DA00037B1613200001213463605801311F43104801195FA310000151000320180109468
:201DC000103200001428CD310000383946360180393AD63102803A3BE03103803BBCEA3102
:201DE00000003C281F3200003132C931E40432B347320000330016320000F10619EBFD0612
:201E0000A9EB131B03C3000033C3221B86C30000C2C39B1B03AA000033AA071C86AA0000A6
:201E2000B6AAEE1A0391000033910F1B86910000B6910B1C037800005778411B867800008F
:201E4000CE78171B035F0000335F1B1B865F0000DA5F631B034600003F46121C864600007C
:201E6000CE46231C032D0000392D771B862D0000C22D8E070314244750524D432C0014D0EC
:201E800011241FBECFEFD8E0DEBFCDBF17E0A0E0B1E001C01D92AE3CB107E1F70E94A82A2B
:201EA0000C94323B0C9400002227E0E0F1E03DB74EB72193E317F407E1F7089584B18F6060
:201EC00084B987B18F6087B98AB188638AB95D9A5B9A579A5C9A5F980895682F690D5B988E
:201EE00065B9629568B95C985C9A672F6A0D5B9A65B9629568B95C985C9A5D985D9A089517
:201F0000672F690D5B9865B9629568B95C985C9A682F6A0D5B9A65B9629568B95C985C9A7F
:201F20005D985D9A0895809146068823B9F098E09924AA248091510770915A0420910305E3
:201F400030916E07D8D080910505709166042091030730911005CFD09A9551F708959CE05D
:201F6000A7E4B6E03FD092E04AD0A0917804B09179041196A0937804B09379040895EDE3B7
:201F8000F2E09924AA249AD0A0917804B09179041196A0937804B0937904089590915804DF
:201FA000A4ECB4E0ED91FD919D90970CAD90A80C0E2E0F2A09F082D09A95A1F7B4DFA4EE84
:201FC000B4E095E00FD0A8EFB4E092E018D0A0917804B09179041196A0937804B093790413
:201FE0005F980895ED91FD919D90970CAD90A80C0E2E0F2A09F0C8D09A95A1F70895ED9198
:20200000FD919D90970CAD90A80C0E2E0F2A09F0B2D09A95A1F70895A7E4B6E09EE1E2DFBC
:2020200091E0EDDFA0917804B09179041196A0937804B09379040895A5E8B4E090910205FC
:20204000DF93CF93C7EDD6E0ED91FD919D90970CAD90A80C0990002009F48DD09A95A1F79B
:20206000CF91DF9190914506992331F0A0916404B091650491E0C3DF809161049927972CF8
:20208000A82CA0E0B1E0880F991F880F991FA80FB91F9091C204992339F08D917D912D9178
:2020A0003D9129D09A95C9F7A0917804B09179041196A0937804B09379040895859188238B
:2020C000E9F38B3071F075912591222309F4F6CF2F3F81F035913F932F930DD08F917F91FF
:2020E000F3CFA5908591292D58D0922E85918F3F09F0E5CF0895AF01EDE6FFE0532E571A13
:2021000008F45194422E481A08F44194451440F4E0E8FFE08727782787272327322723271F
:20212000281730F4822728278227732737277327422E481A532E571A08F4519422243324C7
:202140006624731710F4639401C06A94281780F05F9A0995250C311C022C020C0414310464
:202160001CF0760D24183108839511F0281788F75F98FA01089561E060936304819188239D
:2021800011F00BD0FBCF089561E0609363048591882311F002D0FBCF08952F0187FD59C099
:2021A000815208F456C0482F5527440F551F440F551F440F551FE5EDF4E1E40FF51F68E0FC
:2021C0001F9360906304662021F149B14F77342F3F7D542F577E142F1F7EFF93EF9365903E
:2021E000772767FC4BD071E066FC48D072E065FC45D073E064FC42D074E063FC3FD075E054
:2022000062FC3CD06A9559F7EF91FF9168E01092630449B14068342F3F7D542F577E142F48
:202220001F7E6590662091F0772767FC2BD071E066FC28D072E065FC25D073E064FC22D011
:2022400074E063FC1FD075E062FC1CD06A9549F71F915F98F201893111F488E00DC08038B8
:2022600011F484E009C08C3011F48AE005C08B3011F486E001C08CE0980E089503D07F91C3
:202280007F91C2CF062E770F790D372E3294660F6A0D262E229475B938B85BB94BB965B9E8
:2022A00028B81BB94BB93BB94BB97395372E329475B938B85BB94BB965B928B81BB94BB92F
:2022C0003BB94BB97A95372E32946395262E229475B938B85BB94BB965B928B81BB94BB9BE
:2022E0003BB94BB97395372E329475B938B85BB94BB965B928B81BB94BB93BB94BB9602D22
:202300000895282F3AE1839F1A943AE0812D839F112420192A3010F02A5083950895F1DF2D
:202320008A300CF081E08295822B08950E94302281E30E949321FC016624552482E5282EBA
:2023400087E2382E44245B985D985F9A1BB1012F0F7E520C631CE41D008005B8029408B86B
:202360000BB91BB9F6CF622D732D842D99270895262E372E482E08958AE0280E311C411CAD
:20238000089584E6280E311C411C08959AE0F9DF9A95E9F787E0280E311C411C089594E6FA
:2023A0009F93F4DF9F919A95D9F7822D8951282E31084108822D8A50282E3108410808958A
:2023C000822D8456282E3108410808959AE0F8DF9A95E9F7822D8750282E310841080895A4
:2023E00094E69F93F3DF9F919A95D9F785E2280E311C411C08955A9A80917D07882311F413
:2024000082E001C083E0809369000895E89808951F920F920FB60F9211248F939F938091AE
:202420005B048823F1F080917A07882399F080912D0390912E03019790932E0380932D0329
:20244000892B79F4809127039091280390932E0380932D03F29A10920407809102078093D7
:2024600062049F918F910F900FBE0F901F90189514BC85E085BD8FE787BD0895F19A109244
:202480000103109232038FEF8093340380930303109233031092020382E085BB80936E00DE
:2024A000089510926E0008950F93FC018081882359F081508083882339F4002329F48EB311
:2024C000822B8EBB118213829281990F928383B1862311F0916092838281803841F4818138
:2024E000882399F581E081838DE780832EC08F3789F48381882329F013828EB3209582239E
:2025000005C08181882319F08EB3842B8EBB118210821BC08823C9F485818823B1F08EB30C
:20252000822399F08381882331F491E091838FE0848393830AC0848181508483882329F419
:202540008EB3842B8EBB8FE084830F9108951F920F920FB60F9211240F932F933F934F938A
:202560005F936F937F938F939F93AF93BF93EF93FF9316BC789481E093E060E148E020E13D
:2025800000915D0791DF82E393E060E240E220E400E08ADF809134039091030389238F3F64
:2025A00011F4F1987EDFFF91EF91BF91AF919F918F917F916F915F914F913F912F910F9130
:2025C0000F900FBE0F901F90189510922A0310922903109239041092380410928500109271
:2025E0008400EFE6F0E08081826080830895EFE6F0E080818D7F8083089584E080938100E5
:2026000086E195E09093890080938800DECF3FB7F8942CE3829FC001112490932A038093DF
:2026200029033FBF089580E19EE090933904809338041092C30608951F920F920FB60F9285
:2026400011242F938F939F932BB15F9810928500109284008091290390912A03009729F0D4
:20266000019790932A03809329038091380490913904009751F00197909339048093380469
:20268000892B19F481E08093C30680916204882361F0815080936204882339F481E0809333
:2026A000E806809102078093620480916B04815080936B04882321F4F79A8FE080936B0484
:2026C00080915007882329F08091500781508093500780915B048823E9F090915E048091A3
:2026E0006804891790F480910A05863048F0809104078C3328F481E080935F0710920A05BA
:2027000080910A058F5F80930A05809104078F5F809304078BB12078282B2BB99F918F9106
:202720002F910F900FBE0F901F9018951092B20082E087BB809370000895E0E7F0E08081C2
:202740008D7F808308951092B00087E08093B10081E68093B3000895569A5E980895882358
:2027600011F05E9A08955E98089580917607882309F44E9A089584B18F7C84B985B18063DF
:2027800085B90895F999FECF92BD81BDF89A80B50895F999FECF92BD81BD60BD8FB7F89433
:2027A000FA9AF99A8FBF08959C0180915D07882311F4C901EECF0895A89584B7877F84BF60
:2027C000E0E6F0E0808188618083108208954FB7F89490E0BC01660F771F680F791F9B01D2
:2027E00028593F4FF901859194919093C5008093C40066597F4FFB018491882321F080916B
:20280000C000826003C08091C0008D7F8093C0004FBF08951092C00098ED9093C10096E0B7
:202820009093C200D4DF81E080932F0308951092C0001092C1001092C20010922F03089523
:202840001F920F920FB60F9211248F939F93EF93FF939091000380913103891721F481E0A4
:2028600080932F030BC0E92FF0E0E95FFC4F80818093C6009F5F9F7190930003FF91EF91AF
:202880009F918F910F900FBE0F901F9018951F920F920FB60F9211242F933F938F939F93AC
:2028A000EF93FF933BB15F98909130039F5F2091C60080912C03891751F491E09093520746
:2028C000809181078823A9F09093570712C0E0913003F0E0E85CFC4F2083F09A2A3039F411
:2028E00080918107882319F081E0809357079093300380910C05882339F080915C0788234E
:2029000019F482E0809370008BB13078382B3BB9FF91EF919F918F913F912F910F900FBE2E
:202920000F901F9018951F93182F80912F03882399F4909131039F5F9F7180910003891711
:2029400081F46623B1F0E0917107F0917207099580912F038823B9F310922F031093C60080
:2029600008C0E0913103F0E0E95FFC4F1083909331031F910895CF93DF93EC0102C061E08C
:20298000D2DF89918823D9F7DF91CF910895CF93DF93EC0103C061E0C6DF2196FE0184914F
:2029A0008823C9F7DF91CF910895F09BFECFE0912C03F0E0E85CFC4FE08180912C038F5F59
:2029C00080932C039091300380912C03981709F4F0988E2F0895DC013FB7F8942091300350
:2029E00090912C0380E0E92FF0E0E85CFC4FE0819F5F8F5F681708F0ED93EA3011F0291711
:202A000091F711971C92291709F4F09890932C033FBF0895F09B17C03FB7F894209130035E
:202A200090912C03E92FF0E0E85CFC4F80819F5F8A3019F02917B1F702C0291709F4F0989E
:202A400090932C033FBF0895109231031092000380912F038823E1F3089578940E94E12BF5
:202A6000F894809160008861809360008AE080936000FFCF1F920F920FB60F9211242F93A3
:202A80003F934F935F936F937F938F939F93AF93BF93EF93FF931092B20080910C0588235F
:202AA00011F00E94F821FF91EF91BF91AF919F918F917F916F915F914F913F912F910F905B
:202AC0000FBE0F901F90189590D6E89A0895E2E2F2E0E80FF11DE4918E2F0895FC0185813C
:202AE000882319F483E6858302C08150858385810895FC0180818F5F8C3308F080E0808369
:202B00000895FC0181818F5F8C3308F080E081830895FC0182818F5F883108F080E082836F
:202B20000895FC01862F81508C3008F061E06483862F0895FC0164816F5F6483F2CFFC01F2
:202B4000643608F060E06583862F0895FC0165816F5F6583F4CF8C3310F080E0089580933E
:202B60006C0408958C3310F080E0089580936D040895883110F080E0089580936E04089593
:202B8000FC01262F643658F4862F6AE00E94373A805D8193822F0E94373A905D91938E2F68
:202BA0009F2F08950F931F93CF93DF93EB016B81E7DFDC019DE29C93EC81E150F0E0EE0FEE
:202BC000FF1FEE0FFF1FAF014D575F4FFA01849111968C9311979A012F5F3F4FF901849176
:202BE00012968C931297FA013296E4911396EC93139714969C93149782E315968C931597FC
:202C000080E316968C931697CD0107966D81B8DFDF91CF911F910F9108956CE674E0C2CFF5
:202C2000FF920F931F938B01FB016281A9DF0F2EFAE3FF2EF02DFC01F192CF01F80161812D
:202C40009FDFFC01F192CF01F801608199DF1F910F91FF9008956CE674E0E2CFFF920F934E
:202C60001F938C01F62E862F82958F7030DFF80180838F2D8F702BDFF80181830E5F1F4F7E
:202C8000802F912F1F910F91FF900895282F22952F709AE0299F900111248F70820F089567
:202CA000DC011496EC911497E150F0E0EE0FFF1FEE0FFF1FEA57FF4F84918C3151F41596DD
:202CC0008C9190E083709070892B11F48DE108958CE10895CF93DF93EC018B8181508B83FA
:202CE000882361F48C8181508C83882321F48CE08C83CE01F3DECE01D3DF8B83DF91CF91AD
:202D000008951F93162F662321F0CADF811708F410E0812F1F9108951F93CF93DF93EC01E8
:202D2000162FEFDF882309F411E01B83812FDF91CF911F910895FC0163816F5F6383ECCF2C
:202D4000CF93DF93EC01F7DF813031F4CE01F2DE813011F4CE01FADEDF91CF910895E3EDCD
:202D6000F6E080818F5F8083883120F01082CF010297E6CF08951F93DC0115962C911597D2
:202D8000822F6CE00E94373A592F14963C911497832F90E087509F4FFC01149113964C916A
:202DA000822F90E083709070892B29F4832F8150823008F44150822F6CE00E94373A252F08
:202DC00030E0280F311D2A5F3F4F852F86958695B901680F711DCB0167E070E00E94573A08
:202DE00090E0810F911D67E070E00E94573A90E0840F911D67E070E00E94573A1F91089593
:202E0000EF92FF920F931F937C01862F90E009966CE070E00E94573AE82F6AE00E94373AC8
:202E2000E81AF108042F10E0015010408DE691E09C01E29EC001E39E900DF29E900D112491
:202E4000080F191FC7019695879596958795080F191FC70160E971E00E94433A060F171FB2
:202E6000F0E082E391E09C01E29FC001E39F900DF29F900D112405966AE070E00E94573AE3
:202E8000060F171FC70164E670E00E94433A061B170B20E030E0602F712F822F932F1F91C1
:202EA0000F91FF90EF900895882399F080915E04E82FF0E0E770F070EC5EFD4FE49186955C
:202EC00086958695A4EAB7E0A80FB11D8C91E82BEC9380915E048F5F80935E0408950F934E
:202EE0001F93082F882331F010E080E0DDDF1F5F1017D8F31F910F91089581E0D5DF80E03F
:202F0000D3CF81E0D1DF81E0CFDF81E0CDDF80E0CBCF0F931F93CF93DF9395E0899FC00162
:202F200011248C010E5F184FC0E0D0E0F801EC0FFD1FE491EE2311F0E4DF01C0DEDF21961C
:202F4000C530D10599F7DF91CF911F910F910895813829F4D6DFD1DFD4DFCFDFD2CF823862
:202F600031F4CFDFCEDFCDDFC8DFC7DFC6CF089510925E041092680410920A058BE1E4EAA9
:202F8000F7E0DF011D928A95E9F70895EF92FF920F931F938091A3078F5F8093A3078631AC
:202FA00009F057C01092A30780917607813009F050C00E94EB22882309F04BC0D9DF81E8EE
:202FC000C7DF86E08CDF0F2EFEE6EF2EF4E0FF2EF02DF70180816AE00E94373A9ADF82E0ED
:202FE0007EDFF70180816AE00E94373A892F91DF86E075DF82E8ACDF86E071DFF701829186
:203000008F016AE00E94373A84DF82E068DFF80180816AE00E94373A892F7BDF86E05FDFAA
:2030200082E896DF86E05BDF8EEF9FEFE80EF91EF70180816AE00E94373A6BDF82E04FDFC9
:20304000F70180816AE00E94373A892F62DF86E046DF1F910F91FF90EF900895CF93DF93C7
:20306000EC01442311F4FC0113C083E0683E780710F0FE0103C0FE0180E381936436710557
:2030800010F480E381936A30710510F480E38193CB01BF014AE050E00E940E3BEC2FFD2F12
:2030A000DF010D900020E9F71197AE1BBF0B9E012A0F3B1F822F932FDF91CF910895BF92F5
:2030C000CF92DF92EF92FF920F931F93DF93CF93CDB7DEB769970FB6F894DEBF0FBECDBF84
:2030E000B82E998F6B01C801A0E0B0E08D8B9E8BAF8BB88FC901A0E0B0E0898B9A8BAB8B72
:20310000BC8BCA01A0E0B0E08D879E87AF87B88BBC01CD0120EA35E140E050E00E94183AEC
:20312000EE24FF2487017601E60EF71E081F191F69897A898B899C8920E83CE140E050E050
:203140000E94183AE60EF71E081F191F6D897E898F89988D20E932E040E050E00E94183A7A
:20316000A8019701260F371F481F591F29873A874B875C8769897A898B899C8928E135E230
:2031800040E050E00E94183A7B018C016D857E858F85988926E030E040E050E00E94183A5E
:2031A000E60EF71E081F191F6D897E898F89988D27EF3DE140E050E00E94183AE60EF71EEC
:2031C000081F191F69857A858B859C8520E137E240E050E00E946A3AD801C701820F931FDE
:2031E000A41FB51F8D839E83AF83B8876D897E898F89988D2DE832E140E050E00E94183AF0
:203200007B018C0169897A898B899C892AE230E040E050E00E94183AE60EF71E081F191FAF
:203220006D817E818F81988520E137E240E050E00E946A3AD801C701820F931FA41FB51F49
:2032400089839A83AB83BC83BC01CD0120E137E240E050E00E946A3A69017A016D897E89BB
:203260008F89988D29E131E040E050E00E94183AC60ED71EE81EF91E0B2D198D84E2D801AF
:203280008D938D01C701B60120E137E240E050E00E946A3A9B01AC01C801B90140E0DEDEA9
:2032A0008C0169817A818B819C8120E137E240E050E00E946A3A9B01AC01C801B90141E0D6
:2032C000CDDE8C016D817E818F81988520E137E240E050E00E946A3A9B01AC01C801B90120
:2032E00041E0BCDE8C0169857A858B859C8520E137E240E050E00E946A3A9B01AC01C801A6
:20330000B90141E0ABDE69960FB6F894DEBF0FBECDBFCF91DF911F910F91FF90EF90DF9066
:20332000CF90BF900895BF92CF92DF92EF92FF920F931F93DF93CF93CDB7DEB7AF970FB6C1
:20334000F894DEBF0FBECDBF9E8F8D8F78A36F8FDC0115968C91159790E08053984F149664
:203360006C91149713964C914BDD7B018C018DEC97E06CE04FE144DDAB01BC01E416F50603
:203380000607170720F4EF8DF8A110826CC1AD8DBE8D12969C9112978CE3989F90011124AB
:2033A00011968C91280F311DC901A0E0B0E089A39AA3ABA3BCA3B701641B750B80E090E04D
:2033C00020EA35E040E050E00E94183AE9A0FAA00BA11CA1E60EF71E081F191FA801970155
:2033E00060E070E080E090E0EDA23EA34FA358A769A77AA78BA79CA70F2EF9EDAF2EF02D49
:20340000BB246894B2F80F2EFCE1CF2EF02DDD24EE24FF2400E010E00E942539182F022F75
:20342000085AE1E0021708F0E0E0B32FB65421E0B31708F020E0EB0F31E0EB1708F030E0D4
:20344000232BBE2FA42FAC5431E0A41708F030E0422F4A0F21E04A1708F020E0322BA42F36
:20346000F52FFD5121E0F51708F020E0432F4F0F31E04F1708F030E0232BF42FE62F31E0EF
:20348000661708F030E0422F4E0F21E04E1708F020E0322BE42F572F5B5F41E0571708F044
:2034A00040E0350F21E0351708F020E0422B532F212F81E0111708F080E0420F31E0421788
:2034C00008F030E0832B602F7B2FBF2F0E2FF52EE42ED82ED90E6D8B7E8BAF8BF88FE98F76
:2034E0005A8F4B8FDC8E80918C0790918D0790FF7CC0ED8DFE8D808190E02CE837E7A90129
:20350000849F9001859F300D949F300D1124C901990F880B982F982FE82FC82E8DA78EA7E8
:203520008FA7B62EB20E51E0B61608F050E0272F230F41E0271708F040E0652F620F51E057
:20354000621708F050E0452B262F1A2F190F51E01A1708F050E0642F610F41E0611708F076
:2035600040E0542B162FFB2FFE0F41E0FB1708F040E0652F6F0F51E06F1708F050E0452B84
:20358000F62FE02FEC0D51E0E01708F050E0642F6E0F41E06E1708F040E0542BE62F7DA52A
:2035A0007F0D41E07F1508F040E0652F670F51E0671708F050E0452B762F8EA58E0D91E07D
:2035C0008E1508F090E0542F580F41E0581708F040E0942B8FA58D0D890FBD8A2E8B1F8B7F
:2035E000F88FE98F7A8F5B8F8C8F6D897E894F89588D298D3A8D0B8D1C8D7E010894E11C2E
:20360000F11CC7015CDDF70101900020E9F73197EE19FF093E2F31502E2F2D5FEF8DF8A150
:20362000E20FF11D118240E087015CE2EF8DF8A1E20FF11DD801A30FB11D8C918083315004
:203640003F3F89F021504F5F842F63E00E94373A992361F7332351F3EF8DF8A1E20FF11D89
:2036600050832150E3CFAF960FB6F894DEBF0FBECDBFCF91DF911F910F91FF90EF90DF902B
:20368000CF90BF900895DF92EF92FF920F931F93CF93DF93C3E7D7E000E010E0DD240F2EC5
:2036A000FDE8EF2EF7E0FF2EF02DC8016BD88F3F09F48D2D88830F5F1F4FCE15DF0511F0A7
:2036C0002196F3CFDF91CF911F910F91FF90EF90DF900895EF92FF920F931F93CF93DF93FD
:2036E00003E717E0C0E0D0E00F2EFEE8EF2EF7E0FF2EF02DCE016FEF57D8F80111928F01B0
:203700002196EE15FF05B1F7DF91CF911F910F91FF90EF9008950C94CA38EF92FF920F9322
:203720001F93F82EE62E1FEF82EA0E94D038882319F00E94F73814C08F2D0E94FF388823E0
:2037400019F00E94F7380CC08E2D0E94FF38082F882319F00E94F73803C00E94F73803C01C
:20376000115011F706C0802F1F910F91FF90EF90089581E0809356070FEFF5CF80915D0768
:203780008823D9F480916C048C3328F40E948F11682F82E0C2DF80916D048C3328F40E947A
:2037A0008F11682F83E0B9DF80916E04883128F40E948F11682F84E0B0CF08951F93809163
:2037C0007A07882319F061E010E802C060E411E88FE0A3DF8EE0612FA0DF81E061E19DDFEF
:2037E0001F9108958DE060E098CFFCDFE7CF8DE060E893CF0F931F93CF93DF93EC011FEF9D
:2038000082EA0E94D038882319F00E94F7382BC082E00E94FF38882319F00E94F73823C07F
:203820000E94F73883EA0E94F638082F882319F00E94F73818C00E94113988830E94113903
:2038400089830E9411398A830E9411398B830E9411398C830E9411398D830E941B398E836B
:203860000E94F73803C0115059F606C0802FDF91CF911F910F91089581E0809356070FEF03
:20388000F5CF1F93DF93CF93CDB7DEB727970FB6F894DEBF0FBECDBFCE010196ABDF182F89
:2038A0008F3F09F440C0898188230CF428D789818F77ECD98C3308F080E080936C048A810F
:2038C0008F77E4D98C3308F080E080936D048B818F73DCD9883108F080E080936E048C8124
:2038E0008F73D4D9803208F081E080936F048E818F71CCD9982F81508C3008F091E09093F4
:2039000070048F81C3D9182F843608F010E0E1E7F4E010833597CF016381F3D9882319F46B
:2039200081E080936F04812F27960FB6F894DEBF0FBECDBFCF91DF911F9108951F9380910C
:203940005D07882309F5EFE6F4E01081CF010397612FD7D9882339F0812F0E948F11682F19
:2039600085E0DBDE01C08DDF809170048D3028F40E948F11682F87E0D0DE809171040E9488
:203980008F11682F88E0C9DE1F9108950F931F930EE614E0F801108210926D040250104018
:2039A000F8011082EBDE81E0F801848383831582C5DF85E090E061E00E94D4131F910F9122
:2039C0000895EEE6F4E08081815080838F3F31F487E18083CF0102977DD9B0DFCFCEEEE6B0
:2039E000F4E080818F5F8083873128F01082CF010297A6D9A3DFC2CEFC0180917E07823060
:203A000021F085818551873008F08FEF08951F93162FF2DF982F8F3F11F480E00DC011301F
:203A200019F480917F0705C08091800702C0915086959923E1F781701F910895CF93DF9321
:203A4000EC01DADF8F3F59F18C81833040F1833071F49B8180915C04981708F1981709F5BD
:203A600020E09A8180910B059817E0F01AC0909157048917B0F0891791F49B818091080794
:203A8000981778F0981759F48A81823040F410925904882331F081E08093590402C020E0C4
:203AA00001C021E0822FDF91CF910895CF93DF93EC01A2DF8F3F99F0909157048C81981755
:203AC00080F0981761F4909108078B81981748F0981729F420E08A81823020F002C020E0F4
:203AE00001C021E0822FDF91CF9108951F93162F83DF8F3F11F480E01BC0E82FF0E0EC5E4E
:203B0000FD4F8491113041F460917F07682B60937F078CE090E007C060918007682B6093AA
:203B200080078DE090E00E94D4130E942A2E81E01F9108950F931F93CF93DF938B016115C6
:203B4000710519F4CFE1D0E002C0C1E0D0E0809381040115110511F48AE001C08BE08093FD
:203B60008004C0937F048CE794E005D990E0012B19F0009719F02796C81BD90BCE01DF911E
:203B8000CF911F910F9108950F931F93CF93DF938B016115710519F4CFE1D0E002C0C1E068
:203BA000D0E08093810483E080938004C0937F048CE794E0E0D890E0012B49F0009719F0D9
:203BC0002796C81BD90B9E01295F3F4F03C09E01281B390BC901DF91CF911F910F9108953C
:203BE000CF93DF93EC0110920B0510925C04109208071092570400DF8F3F59F180917E0715
:203C0000882391F482E080930B058BE0809357048D8190E061E070E0B7DF80935C048D81F0
:203C200090E061E070E012C0813099F480930B058AE0809357048D8190E060E070E0A4DFE7
:203C400080935C048D8190E060E070E073DF80930807DF91CF91089581ED96E0C1DF81ED10
:203C600096E0ECDE882391F080915904882311F481E0089581ED96E062E0C9DE882331F41F
:203C800081ED96E062E032DF80E0089580E008951F93182F8CE694E0A3DF8CE694E0CEDE00
:203CA000813079F48CE694E061E0B1DE882309F5112309F094DE8CE694E061E017DF11E0DA
:203CC000E9CF8CE694E0F2DE882399F08CE694E061E09DDE882369F08CE694E062E097DEFF
:203CE000813039F0112329F06CDE8CE694E062E0FDDE1F91089581E0CBCF80E0C9CF10926E
:203D0000C00410928204809107078C7F809307070895DC01FC0180E061936F5F67FD60E22D
:203D20008F5F8431C9F754961C92862F0895E5E8F4E0A1E1B5E08DEE27E09FEFB183A08317
:203D400022838383825155969C93559734965696813FA1F70895FC01DC0180E090E29D9358
:203D60008F5F8431E1F7148A9F012A5E3F4FC90108950F931F93CF93DF936091850470916A
:203D8000860480910205282F30E02150304040E014C01196CB57DB4FFD01EE0FFF1FEE0F3C
:203DA000FF1FEB57FB4F8081918199838883A952B94F8C91F80180834F5FA42FB0E0ED0104
:203DC000CC0FDD1FCC0FDD1F8D010952194FA217B307FCF2CB57DB4F79836883CB01BBDFEA
:203DE00081E0F8018083DF91CF911F910F9108950F931F9321E135E010E001E009C0C901DA
:203E0000AADF9C01E12FF0E0E952F94F00831F5F80910205181798F372DF1F910F91089508
:203E2000E82F80910205E81708F0E0E0F0E0EE0FFF1FEE0FFF1FEB57FB4F8081918108955A
:203E40009091C0049F5F9093C00480910205981738F08FDF8091020581508093C0040AC0B1
:203E6000892FDEDF78DFE091C004F0E0E952F94F81E0808310928204809107078C7F809325
:203E8000070708951F93182F8091070780FF01C0D7DF8091070781FF05C08D7F80930707D8
:203EA000109282048091C004BBDF20918204FC01E20FF11D1083103231F0E091C004F0E03D
:203EC000E952F94F1082809182048F5F80938204843128F0809107078160809307071F9111
:203EE0000895813F69F4862F90E0840F911D813891050CF040E0609361044093C2040895A9
:203F0000823F91F4643118F46093820402C01092820480910205481710F44093C004809134
:203F200007078C7F809307070895CF93DF93EB01E881E7FD17C0F0E0EE0FFF1FEE0FFF1FC0
:203F4000DF01A050BF4F89818C938A81809511968C931197EE5FFE4F8B8180838C81809501
:203F600013968C93DF91CF910895833F61F490E0611191E0990F990F809107078B7F892B75
:203F8000809307070895843F09F5809107078860962F91709295907F8F7E892B80930707BD
:203FA000662331F4109245068EE080930205089581E0809345068DE0809302058091C00426
:203FC0008D30E0F08CE08093C0040895853F89F4809107078062962F91709295990F990FF5
:203FE000907C8F7B892B80930707662309F425C314C3863F19F4662309F4FACE089583E869
:2040000094E00C94BD381F938091830490918404892B99F51091C004812F02DFDC01E1E4CA
:20402000F4E08D9181938823E1F7E0918204E43110F0E3E106C08091070780FF02C0E1110F
:20404000E150F0E0EF5BFB4F8FE58083812F90E0880F991F880F991F8B579B4F6FEF41E447
:2040600054E00E942C389093840480938304E091C004F0E0E952F94F10821F9108950F93B8
:204080001F9301E115E0C80161EF76E00E94D73AF80101900020E9F73197E01BF10BCF015C
:2040A000800F911F66E071E00E94D73A1092D70681E08093C00461E308E016E10DC0019F30
:2040C000C00111248F5E9A4F24DE682FE02FF0E0E952F94F10820F5F80910205081778F377
:2040E0001F910F9108950BDE109261041092C20410923F0480910707846087788093070773
:2041000080918C0784FF02C08EE001C08DE0809302050DDE6DDEB3CF1F930E94D514182FC4
:2041200080913F04813051F4173FE8F410932B0382E080933F041092400474C0823069F550
:2041400080914004E82FF0E0E65CFB4F10838F5F80934004813051F480912B03833F08F4CC
:2041600061C0612F02DF10923F045CC0823051F480912B03813F08F455C060913A04412F06
:20418000B0DEF1CF853009F04DC080912B03803F51F76AE374E0C9DEE6CF1F3F31F481E0EF
:2041A00080933F0410922B033DC01032B8F5183041F4809182048823A9F18150809382042A
:2041C00031C01D30A1F48091070781FF01C038DE9091070790FF07C080918204843110F1C4
:2041E0009E7F909307078091070782600FC0193011F480E216C01A3061F48091070780FFDE
:2042000001C01EDE8091070781608D7F8093070709C08EE537DE812F8F5B03C017FD02C030
:20422000812F30DE1F9108958091070783FF09C084FF0BC081E0809345068DE08093020575
:2042400015C080918C0784FF04C0109245068EE0F5CF81E0809345068DE080930205809128
:20426000C0048D3018F08CE08093C00480918C0785FF10C088EF94E0909365048093640488
:204280008091F8049091F90487D18093FA041092FB0408C08CEF94E090936504809364042B
:2042A0001092FF048091070785FF03C086FD06C0C4C180918C0786FD01C0BFC108950F937E
:2042C0001F938CE190E19093720780937107ACDF82E48093500702E4FDD6F59B03C08FDE53
:2042E0000E94A129F39B07C0F39889DE96D1C7D51F910F910895F09B0AC081DE1FEA0CDF73
:20430000F09B02C01150D9F700935007E5CF80915007882309F78091070782FF01C073DEBC
:2043200010923F04D9CF20E131E0A0E0B1E040E09EEF813329F4F9012F5F3F4F949114C040
:20434000823311F4942F10C0833349F447FD02C09E5F0AC0403809F491E0925005C084330C
:2043600019F4942F990F990B9C934F5F51E0AF3FB50711F01196DDCF80E091E008950C9407
:204380002D150F931F930E94D5140E94D514082F0E94D514182F0E94D514682F712F802FF7
:2043A00090E00E94B8111F910F910895FF920F931F930E94B311F62E072F182F80E593EC65
:2043C0000197F1F786E40E94E82B80E00E94E82B812F0E94E82B802F0E94E82B8F2D0E9402
:2043E000E82B8AE00E94E82B1F910F91FF9008950E949D1381E080935C071D9902C00E94CC
:204400002D1578940E94D5148D3219F40E94BC111EC0843619F40E94C61119C0843419F4CC
:204420000E94CF1114C08B3219F40E94DA110FC0853719F40E94E6110AC0853519F40E946B
:20444000F01105C0833711F49CDF01C06CDFAEDF80912F038823E1F3F89410925C070895D3
:204460000E94E12BF8940E9406120E9451120E94F7120E949D1384E00E94E71381E08093D2
:204480000C057894089581E0089581E008958FEF80930303809334038093550788E2809399
:2044A00009078FE48093C30488E08093580484E397E09093C5048093C4041092040581E017
:2044C000809354078EE380930207809362048FE080936B0484E18093A30708951092CA0448
:2044E00080917C07843019F420E030E021C0833031F483E58093CA0421EB34E119C080914A
:204500007B07853021F0833011F0843069F4209100053091010580916E048C3048F02091E9
:204520006F073091700704C020910005309101053093C9042093C804089580917B07863097
:2045400010F010927B0780917B07089580917C07863010F010927C0780917C070895809156
:204560008307853010F4823011F4109283078091830708958A3311F488E00895803811F459
:2045800084E008958D3211F48AE008958C3211F08CE0089586E008950F931F93CF93DF935C
:2045A0008C01C0E0D0E003C0E5DFC80FD11DF80181918F018823C1F7CF3FD10509F030F4D3
:2045C0008FEF90E08C1B910995958795DF91CF911F910F91089580910405811181E00895FF
:2045E0001092620408958091020780936204089580915E07882381F48091C1048F5F877095
:204600008093C104E82FF0E0EE0FFF1FE959FC4F85919491782E892E0895809179078530B8
:2046200059F010925E0790E005966AE070E00E94573A80936704DCCF089581E080935E07B3
:204640007724882410926704089580917907853009F4F3CFE2CF8091270390912803909309
:204660002E0380932D03089520917A07222349F02F3739F0822F90E027FD9F6F8050904FE8
:2046800002C080E090E19093280380932703089580E097E00C94BD3887E496E06DE174E070
:2046A00048E350E00C94C33A1F931FB7F89480937A0784D8D9DFCFDF96DF1FBF1F910895F8
:2046C000682F80EF94E04EE152E00C942C388091040581FD0CC08091000790910107892BA2
:2046E00031F48FEFEDDF90930107809300070895682F8CEE94E04CE152E00C942C38809170
:2047000055078F3F79F481E08093550780910D0590910E05892B31F480EFEADF90930E0594
:2047200080930D0508951F93182F809387070E942415812F0E94E7131F9108951F938091E6
:20474000E506282F30E040E050E080915D07882311F041E050E0242B352B232B11F5809131
:204760008407882341F480E280938E0710928F0781E08093840781E190E0609184070E949D
:20478000D41310E00AC0E12FF0E0CF014E96E257F84F60810E94D4131F5F809184071817B1
:2047A00090F31F9108951F93682F192F80938C0790938D0789E190E00E94D4138AE190E0FD
:2047C000612F0E94D41380918C0790918D079695879596958795809581708093460681E013
:2047E0001F910895682F8093790786E090E00E94D4132BDF81E00895682F8093770784E04F
:2048000090E00E94D41381E00895682F8093740781E090E00E94D41381E00895FF920F93F1
:204820001F93809184078150843110F4FF2418C08BE0809384078EE897E061EF76E00E9467
:20484000D73A81E08093E50613C00F2D10E0C8014E960E94C2130257184FF8018083F39482
:20486000E0918407FE1688F3F0E0E257F84F10821F910F91FF900895FF920F931F93F82E44
:2048800080918307813029F41092F9041092F80433C0882339F48EE897E09093F904809387
:2048A000F80421C0833091F48CE694E00E94BB16E82FF0E0EE0FFF1FE451FF4F659174910A
:2048C0000AEE16E0C8010E94D73A09C0843059F40AEE16E08CE694E0B8010E949319109326
:2048E000F9040093F8048091F8049091F90454DE8093FA04F092FB041F910F91FF900895C1
:2049000084EA8093CE0482EC8093D2048EE58093D6048CE78093DA0487E18093DE0485E364
:204920008093E20485EAA8DF80E698E09093C5048093C404D3DD80918C0790918D079695AF
:204940008795969587958095817080934606089588EB8093CE048FEC8093D2048EE68093AF
:20496000D60485E88093DA0480E28093DE0487E38093E20489E180DF82E392E09093C504B9
:204980008093C404ABDD109246060895ECECF4E0118210821282349684E0E43EF807C1F7BD
:2049A00081E96ADF84E397E09093C5048093C40495DD1092460608951F93182F8093760719
:2049C00081115E980E94B81784E18093A30783E090E0612F0E94D41381E01F910895682F8B
:2049E00080937D078AE090E00E94D4130E942D1581E00895682F80937E078BE090E00E942F
:204A0000D41379C99C0180917B07823019F4C9010C942E16C9010C94C01580917B0781502D
:204A2000823000F5809104078695982F9695969560910407680F690F96959695690F643628
:204A400008F064568091040580FF03C083E6861B682F8091E6069091E706009719F0D2DF4B
:204A6000FC01108208950F931F93CF93DF9310917B07153019F4C1E6D7E05DC0133031F48A
:204A800081E697E00E940D16EC0155C01430D9F481E697E060918B07B5DF1AE3FC011193CD
:204AA000CF0160918A07AEDFFC011193CF0160918907A8DFFC0180E8808381E481838CE45D
:204AC0008283EF0137C060916E04112329F4E62FF0E0E15BFC4F649181E697E093DF0AE398
:204AE000FC010193CF0160916D048CDFFC010193CF0160916C0486DFEC01112369F480E87B
:204B0000888380916E048C3010F080E501C081E489838DE48A830EC080918607882359F0D6
:204B20001150123040F4FE010193F093E706E093E60673DF2396188281E697E09093FD0495
:204B40008093FC0429DD8093FE04DF91CF911F910F910895682F8093860783E190E00E94BD
:204B6000D41381DF81E0089580937B07E6DC682F88E090E00E94D413B1DC75CF8093BD04FC
:204B800072DF8091BD04882361F1A4ECB6E0E1E6F7E08DE001900D928150E1F78091BD0419
:204BA000823019F4E7ECF6E019C0833019F4EAECF6E014C0853041F480E28093CB06809331
:204BC000CC06EDECF6E00AC0843019F0E4ECF6E005C080E28093C706E8ECF6E080E2808311
:204BE00081830895DF92EF92FF920F931F93CF93DF93082F862F0E948F11D82EC02FD0E096
:204C000082958F70E82FF0E0EE0FFF1F0DE914E1E00FF11F2591349184ECE82E84E0F82E07
:204C2000FE01EE0FFF1FEE0FFF1FEE0DFF1D20833183CF01B9010E946734ED2DF0E0EF70C1
:204C4000F070EE0FFF1FE00FF11F25913491FE013196EE0FFF1FEE0FFF1FEE0DFF1D2083A9
:204C60003183CF01B9010E946734DF91CF911F910F91FF90EF90DF900895CF92DF92EF922C
:204C8000FF920F931F93CF93DF93E82E862F8A0169010E948F11F82ECE2DD0E082958F7072
:204CA000E82FF0E0EE0FFF1FE00FF11F2591349104EC14E0FE01EE0FFF1FEE0FFF1FE00F70
:204CC000F11F20833183CF01B9010E946734EF2DF0E0EF70F070EE0FFF1FEC0DFD1D259117
:204CE0003491FE013196EE0FFF1FEE0FFF1FE00FF11F20833183CF01B9010E946734DF9166
:204D0000CF911F910F91FF90EF90DF90CF90089580917C07833089F480918C0783FF09C0B7
:204D2000E0916E04F0E0E15BFC4FE49186E06E2F03C086E060916E0455CF843041F486E0C2
:204D400060916E044BE652E02BE333E096CF80916E046CE00E94373A85E0989F90011124C3
:204D600080916D040E94373A280F311DB901E3E0660F771FEA95E1F7620F731F60567E4EB5
:204D80007093DD046093DC048CED94E00C94673480917C07833021F484E060916D0422CF21
:204DA000843039F460916D044DEA52E02BE333E064CF60916D0489E0689FB00111246C5778
:204DC000704F7093D5046093D40484ED94E00C94673480917C07833009F02CC082E06091CE
:204DE0006C0400DFE0916C0489E0E89FF0011124E05AF74F8491809351073196849180937E
:204E00005A0431968491809303053196849180936E073196849180930505319684918093F1
:204E2000660431968491809303073196E491E09310050895843041F482E060916C044DEACB
:204E400052E02BE333E019CF60916C0485E0689FB0011124685A714F7093CD046093CC044B
:204E60008CEC94E00C946734B4DF92DF51CF1092530734DBF9DFF7DD8091FB04FDCC1F93A5
:204E800065DB182F843091F489E78093EA0491E09093EB048BE68093EE049093EF0487E863
:204EA0008093F2049093F30453DD44C0833091F489E78093EA049EEB9093EB048BE68093D3
:204EC000EE049093EF0487E88093F2049093F30417DD30C0882319F48CE79AE012C081302C
:204EE00049F48CE79AE090930105809300058AE69BE00BC0823019F48EEC9CE002C084EFA7
:204F00009DE090930105809300059093700780936F0789E78093EA0494EB9093EB048BE63D
:204F20008093EE049093EF0487E88093F2049093F3042CDD9CDF812F1F91089580938307A6
:204F40000EDB682F80E190E00E94D41398CF80937C0795DF682F89E090E00E94D413BEDA75
:204F600083CF39DB882319F40E94411C80CF08951F93182F80910405812781FF09C011FD16
:204F800002C08EE301C082E080936204809302070E94B81784E18093A30710930405E1DF27
:204FA0001F9108958091040581FF05C08EE3809362048093020710920405D3CF0E94B51388
:204FC0000E94C61780916C04815080936C048F3F59F080915307813009F449CFFADE80914C
:204FE000090784FD1DC03FCD2BE320936C0491E090935A0780916D04815080936D048F3F6C
:2050000071F420936D0490935B0780916E04815080936E048F3F19F487E180936E0427CFEB
:2050200008950E94B5130E94C61780916C048F5F80936C048C3388F480915307882309F0AE
:205040003CC080918C0790918D0790FD36C0C1DE8091090784FD3DC006CD91E090935A0772
:2050600010926C0480916D048F5F80936D048C33E0F090935B0710926D0480916E048F5F92
:2050800080936E04883188F010926E048091090784FD04C08CE694E00E94A0168091040588
:2050A00081FF0BC00E947B1E08C08091E806882321F48091040581FF01C0D9CE0E94BE1B66
:2050C0008091090784FD04C00E94411C0E947B1ECECE089580918607882329F08091780408
:2050E000877009F49ADCE0917107F09172070995F19906C083B18073803311F00E943E12A8
:20510000F69B03C0F6980E942D1580915F078823E1F020916804822F90E0877090708C5EB7
:205120009D4FFC019491269526952695E22FF0E0EC55F84F808189230E94AF138091680439
:205140008F5F8093680410925F07F29B7DC08091060590910705A0910805B09109050196A3
:20516000A11DB11D8093060590930705A0930805B09309058091720490917304A0917404FD
:20518000B09175040196A11DB11D8093720490937304A0937404B09375048091040580FF0F
:2051A00002C00CDF01C03DDF80915D0780FF09C081FD01C06DDA80915D0782FF03C018DA77
:2051C00001C066DA80915D04882389F590916E0480918B07981759F590916D0480918A07CC
:2051E000981729F590916C04809189079817F9F4809177078823D9F480915D078823B9F440
:205200008091760490917704892B89F480910907883368F484EC94E060EF40E050E00E94D9
:205220002C3890937704809376040E94131380917804909179049093600480935F0410924D
:20524000790410927804F2988091E806882361F0109204073CDA8091040580FF02C0AEDE84
:2052600001C0DFDE1092E806F79B03C00E948838F7988091290390912A03892B19F481E02D
:205280008093540780915A07882309F43EC080916704815080936704882359F4A9D9809132
:2052A000790790E005966AE070E00E94573A8093670480917407882309F0FDD410925A0714
:2052C00080915B07882309F120E030E080917607833011F421E030E08091740790E0282308
:2052E00039238091770790E028233923232B59F080916E04843039F484EF94E060EF40E15A
:2053000052E00E942C3810925B078091C306882361F08091760490917704892B31F01092DD
:205320007704109276041092C30680915207882339F080917607823009F44E9A109252070D
:205340000895EF92FF920F931F93DF93CF93CDB7DEB764970FB6F894DEBF0FBECDBFF5988E
:205360008091760490917704892B29F086E794E00E94BD386BC0E0907107F09072078CD950
:2053800080915F04909160048E010F5F1F4FB8014AE050E00E940E3BF80101900020E9F721
:2053A0003197E01BF0E0D801AE0FBF1F88E48C93DE01AE0FBF1F8AE712968C931297FD0102
:2053C00013821093780600937706609106057091070580910805909109058E01075F1F4F4E
:2053E000A8012AE030E00E94EB3AF80101900020E9F73197E01BF0E0D801AE0FBF1F83E52A
:205400008C93EC0FFD1F128610937C0600937B068FEA9FE0909372078093710784E00E9460
:20542000071358DE0E940A158091290390912A03892B21F0F39902C0F59BF3CFF59880E07E
:205440000E940713F0927207E092710764960FB6F894DEBF0FBECDBFCF91DF911F910F914A
:20546000FF90EF9008958FEB9FE090937207809371070E94F71B2EDEF59B01C062DFF39B81
:2054800005C0F3980E94F21B80E0089580918107882319F00E941D38EECFF09BECCFB4D441
:2054A000882349F30E94F21B81E008958EEC9FE0909372078093710789E48093FF04109213
:2054C000720410927304109274041092750402DEF59B09C036DF10927204109273041092E7
:2054E000740410927504F39B03C0F39880E008958091720490917304A0917404B0917504BE
:2055000089559240A040B04038F080918C0790918D0791FF01C07AD5F49B0BC0F4980E9462
:2055200033351092720410927304109274041092750480918107882319F00E941D38C7CFC3
:20554000F09BC5CF61D4882309F4B9CF81E00895CF93DF930E94DC1381E0809364001EBAB4
:20556000882477240E9447220E948B1B0E9438120E94FD120E94A3130E945E0F0E94AC132C
:205580005E980E94BB130E9468380E94431B0E949D220E94A6220E94AF220E94FB1164D83B
:2055A0005AD853D83BD980918707893038F01092870784E190E060E00E94D413809187078D
:2055C0000E940A1480918807843030F085E190E060E00E94D41380E080935D040E947320EF
:2055E0000E94B81759D88FEA9FE090937207809371070E94F21B80915607882331F48091EC
:205600007807882311F40E94C61C0E94411C0E94641581E080935B0478940E947B1E2FDC98
:20562000F0D381E0CCE0D0E103C081E001C080E0D0937207C09371070E94EC3518DC809135
:205640005D04882311F432DF03C0813021F40BDF882359F7ECCF823019F40E945F21E7CF68
:20566000833019F40E949611E2CF843011F4CED4DECF8530E1F60E942D15D9CF90E0880F49
:20568000991FFC01E65AFB4F259134918E599B4FFC01A591B4918C9191E08927F901099531
:2056A000089590E0880F991F8E569B4FFC0125913491F90109950895FC0180E28193CF01D0
:2056C0000895982F81568A3108F49052892F0895CF93DF93EC018881982F90539A3040F033
:2056E000603149F4EEDF982F8154863020F49753988381E001C080E0DF91CF91089588E14C
:2057000095E00E94C71481E008958BE295E00C94C714FBDF81EF96E00E94C71486EA94E01B
:205720000E94C7148DEF96E00C94C714F2DF8BE495E00E94C71481E008950F931F93182FB4
:20574000092F6BE275E00E94D73AA12FB02FFD0101900020E9F73197EA1BFB0BE80FF91F9C
:20576000CF011F910F9108950E946A1B0E942D1581E0089580917407882319F00E94411C24
:2057800076DBC7DF81E008951F93CF93DF93EC0180916C04182F125E1C3348F01C5307C0AC
:2057A00099DC80916C04811711F480E006C0F09BF7CF0E94D514888381E0DF91CF911F9168
:2057C000089501C087DC80912F038823D9F3089561E00C949314CF92DF92EF92FF920F93A3
:2057E0001F93DF93CF930F92CDB7DEB782E195E00E94C7140EE817E0FF24EE246E010894E7
:20580000C11CD11CC601C0DF882321F40E94DA3480E03AC08981DCDF9F2D9F5F89818D3038
:2058200089F08A3079F0F80181938F01803211F0EE2404C0EE2041F4EE24E394943121F004
:20584000F92EE0CF2F2D01C0292F8D3049F08A3019F406C091508F01F80182918032D1F387
:20586000222349F480918307882311F481E001C080E064DB08C0F8011082909384071092F7
:20588000E5060E94803481E00F90CF91DF911F910F91FF90EF90DF90CF900895DF92EF923C
:2058A000FF920F931F93DF93CF930F92CDB7DEB77C01D62E8E010F5F1F4FC80165DF8823D1
:2058C00071F0898185DF8981FCDE883541F0C8016D2DFEDE8981F701808381E001C080E061
:2058E0000F90CF91DF911F910F91FF90EF90DF9008950F931F93DF93CF9300D000D0CDB783
:20590000DEB78B010E94C714CE01019660E1C6DF882379F1CE01029660E1C0DF882349F15C
:20592000CE01039660E1BADF882319F1CE01049660E1B4DF8823E9F0298130E064E0220F80
:20594000331F6A95E1F78A81280F311D322F22278B8190E044E0880F991F4A95E1F74C8171
:20596000840F911D282B392BF8013183208381E001C080E00F900F900F900F90CF91DF9111
:205980001F910F910895DF93CF9300D0CDB7DEB78EE295E0BE016F5F7F4FABDF882321F0D7
:2059A00089819A810E94D3230F900F90CF91DF910895EF92FF920F931F93DF93CF9300D075
:2059C000CDB7DEB78C017B0181ED94E00E94C714C8010E94C714CE0101966AE05FDF882367
:2059E00089F0CE0102966AE059DF882359F089812AE0829FC00111242A81280FF7012083A9
:205A000081E001C080E00F900F90CF91DF911F910F91FF90EF9008950F931F93DF93CF93D3
:205A20000F92CDB7DEB78EEE94E08E010F5F1F4FB801BFDF882369F18CE694E069810E9483
:205A40009F159981891729F560DE85EF94E0B801B0DF8823F1F08CE694E069810E949115A8
:205A600099818917B1F451DE8DEF94E0B801A1DF882379F08CE694E069810E948C1699812D
:205A8000891739F40E949E1C0E947B1EF0D981E004C03BDE0E94411C80E00F90CF91DF91CD
:205AA0001F910F9108950F931F93DF93CF930F92CDB7DEB78AED94E08E010F5F1F4FB80108
:205AC00078DF882339F189810E94B9159981891709F51BDE80EE94E0B8016BDF8823D1F01E
:205AE00089810E94B21599818917A1F40EDE87EE94E0B8015EDF882369F089810E94AB15A9
:205B00009981891739F40E94BE1B0E947D1EAFD981E003C00E94411C80E00F90CF91DF916C
:205B20001F910F910895FF920F931F93DF93CF930F92CDB7DEB7F82E8B018FEB94E00E94C3
:205B4000C7148F2D805D44DE89E242DE8AE340DECE0101966AE0A2DE882339F08981F8167D
:205B600020F0F801808381E001C080E00F90CF91DF911F910F91FF900895DF93CF930F9237
:205B8000CDB7DEB785E0BE016F5F7F4FCCDF8823A9F0698180915D04681711F481E00EC02E
:205BA00060935D04623011F0662329F4698385E190E00E94D41381E0809359070F90CF913A
:205BC000DF910895EF92FF921F93DF93CF930F92CDB7DEB7182F282F30E0C901880F991F9F
:205BE0008E589B4FFC01E590F49020583B4FF9018491BE016F5F7F4F96DF8823A1F0123080
:205C000021F48981823051F40EC0163039F48981853010F0855001C08B5F89838981F701E0
:205C2000099581E001C080E00F90CF91DF911F91FF90EF900895FC016193CF01642F0E9484
:205C40002E163ACD66E640917F07F5DF62E640918007F1CF0F931F93DF93CF93CDB7DEB7E1
:205C6000C054D0400FB6F894DEBF0FBECDBF82E495E00E94C7148E010F5F1F4FC801E2DF6C
:205C80005CDDC8010E94BB14C05CDF4F0FB6F894DEBF0FBECDBFCF91DF911F910F91089543
:205CA0001F93142F452FC7DF0197612F0E942E1603DD1F9108950F931F93DF93CF93CDB7EE
:205CC000DEB7CB54D0400FB6F894DEBF0FBECDBFCE0101960E940D16EFDC0E942B16ECDC18
:205CE000182F092F8CE694E00E94BB16E82FF0E0EE0FFF1FE451FF4F65917491812F902FDD
:205D00000E94D73AA12FB02FFD0101900020E9F73197EA1BFB0B8E0F9F1FCEDC6CE4409199
:205D2000760789DFFC0180917407882311F086E5819380917E07882311F485E503C08130A6
:205D400011F485E4819380918607882311F08BE4819380917907853059F090E005966AE010
:205D600070E00E94573A482FCF0162E464DFFC0180910405882311F086E4819380915D041D
:205D8000813011F483E48193CF0196DC5BDF6DE440917D0750DF40918C0750918D0769E45B
:205DA0007FDF282F809177078823C9F4E22FF92F81E48193CF0160918B070E94C0151AE3BE
:205DC000FC011193CF0160918A070E94C015FC011193CF0160918A070E94C015282F822FE7
:205DE000ACDCCE0101960E94BB14C55BDF4F0FB6F894DEBF0FBECDBFCF91DF911F910F918F
:205E0000089587DC82DC57CFEF92FF921F93DF93CF930F92CDB7DEB70E94D51452DC8983E7
:205E2000883521F00E940A1580E051C07E010894E11CF11C8CED96E00E94C714C701A4DC89
:205E4000882309F444C08981C3DC89813ADC182F115419831F5B80E2BBDC89818A3150F706
:205E60001092590795E5E92E94E0F92EC701612F70E00E94CC3A009719F08E19FFDB1BC0A8
:205E80008AE6E82E84E0F82EC701612F70E00E94CC3A009719F08E1995DE0DC0B7E8EB2E63
:205EA000B4E0FB2EC701612F70E00E94CC3A009721F08E19F6DB882321F483E095E00E947B
:205EC000C71423DCF8DE0E943727809159070F90CF91DF911F91FF90EF900895809181073E
:205EE00091E0892780938107882311F48CE301C089E495D781E0089580E029D880E00C94CE
:205F0000B42583E0809383070C943727582F282F392FAEE8B7E0822F851BF9012F5F3F4FD0
:205F2000E491ED93EE23B9F780938407109283070C9437278AE09BE19093E5048093E404F6
:205F400089E68093E6048DE28093E7042BD880E00E94AA258EEC9FE0909372078093710774
:205F600089E48093FF048FE080936E048AE280936D040E943F2781EF96E0C8DFBDCF0E94F7
:205F80000713A8D80E940A158091290390912A03892B11F0F59BF5CFF59880E00C9407136B
:205FA00085E0EDCF83E0EBCF82E0E9CF80E00E94B425FADF83E00E94B425F6DF81E00E941F
:205FC000B425F2DF81E00E94AA25EEDF80E00E94AA2582E00E94B425E7DF80E00E94B42529
:205FE000E3DF85E00E94B425DFDF83E00C94B425CF93DF93EC01FE018491882321F00E9432
:20600000421F2196F8CFDF91CF910895EF92FF920F931F9381E080935D078CDF76DB8CEEC0
:2060200098E10E94C714C2DF8DEC97E16FDF80E00E94A727B7DF85E00E94A727B3DF81E05C
:206040000E94A727AFDF82E00E94A727ABDF89EE97E15CDF83E00E94A727A8DF8CED97E171
:2060600055DF84E00E94A727A1DF8CE298E14EDF82E00E94B42596DF80E00E94A72780E002
:206080000E94B4258CED98E141DF8CDF89E398E13DDF8ADF36DF88DF81E00E94AA2581E0EF
:2060A0000E94A7277FDF80E00E94AA2583E00E94B42578DF82E00E94A72774DF83E00E94E2
:2060C000A72770DF84E00E94A72780E00E94B42569DF85E00E94A72782E00E94B42562DFB9
:2060E00080E00E94B42580E00E94A72781E098E10DDF81E00E94DC2453DF89E498E106DF2F
:2061000053DF8FEB9FE090937207809371074ADF0EEC1FE010937207009371078CE598E1FA
:20612000F5DE42DF3CE1E32E30E1F32EF0927207E092710785E00E94B42581E00E949E277E
:206140002FDF109372070093710780E00E94B42583E798E1DBDE28DFF0927207E0927107A7
:2061600084EF60E00E94B51F85EF60E00E94B51F86EF60E00E94B51F00E010E000933A0400
:20618000C801880F991F880F991FFC01E65AF64EE491E0933B04FC01E55AF64EE491E09388
:2061A0003C04FC01E45AF64EE491E0933D04835A964EFC01849180933E0480EF6AE374E0BF
:2061C0000E94951F0F5F1F4F05361105B9F681EF60E045E60E94711F82EF60E04DE00E9400
:2061E000711F85E698E104DFDBDE84EF61E00E94B51F85EF61E00E94B51F0EEC1FE010939E
:2062000072070093710783E898E180DECDDE99D883E198E17BDEC8DE16D383E596E0D6D44F
:206220008CE090E19093720780937107B9DE109372070093710787EF97E168DE82E00E9464
:20624000B827B0DE0E94D227AFDE81E00E94B827A9DE83E00E94B827A5DE0E94D2278AE0D4
:2062600098E154DE8CE00E9478239CDE83E080935D078CE00E94602395DE01E000935D079A
:206280008CE060E00BD68EDE84EC94E06CE040E050E0E2D687DE8FE898E138DE85E08093EA
:2062A0005D0710915E0710925E071092C10478DE10935E0700935D0781EA98E127DE72DE78
:2062C00080EB98E123DE6EDE81EC98E11FDE6ADE86ED98E11BDE66DE0FDE82E298E116DE7B
:2062E0005FDE0E942D1581E01F910F91FF90EF9008958EE58093C30408958091CA07ECEC7D
:20630000FCE1E80FF11DE4918E2F0895E0917A07EF3711F481E00895EE2311F480E008959E
:20632000EC5FF0E0EA52F34E84910895982F87FF02C0F39A9F7796FF04C081E08093580735
:206340009F7B892F08958AE89BE19093E5048093E4048BE28093E6048DE28093E704089565
:20636000F59A0895F59A08958093C3048AE794E004C78093090789E694E0FFD68EEB94E073
:20638000FCC688E2F6CF83E894E0F7D61092BD040895D9DFF8DFF59A0895F5DF0E949E1C75
:2063A0000E947B1E0E943727F59A089580918B078F5F883108F080E080938B070C94372731
:2063C00080918A078F5F8C3308F080E080938A070C943727809189078F5F8C3308F080E0CE
:2063E000809389070C9437278CE694E00E94A6150C9437278CE694E00E949A150C94372786
:206400008CE694E060916F040E948116882331F48CE694E00E94501680936F04F59A089589
:206420008CE694E00E949B160C9437270E94411CA8DF1092E5041092E4040C943727A3DF0A
:2064400086E190E0609189070E94D41387E190E060918A070E94D41388E190E060918B071C
:206460000E94D4138EDF0C9437276091BF0780915D04681759F060935D04662311F06230C7
:2064800021F485E190E00E94D41333CF08950E94BE1B0E947D1E75DF1092E5041092E404C8
:2064A0000C9437278CE694E00E9489150E94372781E00C94BE258CE694E00E9481150C9416
:2064C00037278CE694E00E9479150C943727AAEEB6E0EEE8F7E085E101900D928150E1F730
:2064E000E091E906F0E0E651F94F8FE5808308958091E906A82FB0E0FD01E257F84FE08193
:20650000EF5FE7FDE0E2A257B84FEC93E0CF2091C0078EE897E0FC01E20FF11D10820E94C4
:20652000CC228093C10608958093C907E82FF0E0EE0FFF1FE851F34E259134912093BB06A8
:206540003093BC0680917A0490917B046BEB76E0A901BFC58091C9078F5F853008F080E0D1
:20656000E3CF482F8093CD0750E0440F551F440F551F4155554E509364064093630680917A
:206580007A0490917B0463E676E0A3C58091CD078F5F863508F08CE3E4CF8093CA07E82F33
:2065A000F0E0EE0FFF1FE854F34E2591349120937B0630937C0680917A0490917B046BE7FE
:2065C00076E0A90186C58091CA078F5F8A3008F080E0E3CF8093BF07E82FF0E0EE0FFF1F01
:2065E000E850F34E25913491209373063093740680917A0490917B0463E776E0A90169C597
:206600008091BF078F5F863008F080E0E3CF8093CC07E82FF0E0EE0FFF1FEC54F34E2591D6
:2066200034912093AB063093AC0680917A0490917B046BEA76E0A9014CC58091CC0791E0D2
:206640008927E5CF8093C707E82FF0E0EE0FFF1FEC54F34E2591349120938306309384066E
:2066600080917A0490917B0463E876E0A90131C58091C70791E08927E5CF8093CB07E82FFA
:20668000F0E0EE0FFF1FEE55F34E259134912093B3063093B40680917A0490917B0463EBAA
:2066A00076E0A90116C58091CB078F5F893008F080E0E3CF8093C807E82FF0E0EE0FFF1F87
:2066C000EE50F34E2591349120936B0630936C0680917A0490917B046BE676E0A901F9C42A
:2066E0008091C8078F5F833008F080E0E3CF8093C607E82FF0E0EE0FFF1FE052F34E259104
:2067000034912093A3063093A40680917A0490917B0463EA76E0A901DCC48091C6078F5F03
:20672000843008F080E0E3CF482F8093C30750E0440F551F4259534E50939C0640939B061B
:2067400080917A0490917B046BE976E0C2C48091C3078F5F8093C3078A3010F01092C3070E
:206760008091C307E1CF8093C207E82FF0E0EE0FFF1FE656F34E25913491209393063093A9
:20678000940680917A0490917B0463E976E0A901A0C48091C2078F5F8093C207843010F028
:2067A0001092C2078091C207DECF8093C107E82FF0E0EE0FFF1FE851F34E25913491209362
:2067C0008B0630938C0680917A0490917B046BE876E0A9017EC48091C10791E08927E5CF61
:2067E0008093C407E82FF0E0EE0FFF1FEE57F34E2591349120935B0630935C0680917A04F0
:2068000090917B046BE576E0A90163C48091C4078F5F863008F080E0E3CF8093C507E82FE1
:20682000F0E0EE0FFF1FE257F34E25913491209353063093540680917A0490917B0463E5D8
:2068400076E0A90146C487E496E06AEF7DE14CE750E099D680917707A8DF80917B07DDDF5F
:206860008091760780DF809179075EDF80917C07B7DF809104053BDF80915D04ABDE8091F3
:20688000830752DE80918607DDDE809184078093C0071092E9063BDE80918107882321F070
:2068A00080918207875B01C08CE35BDE80917E0701DF80E0ACDE80918707DFDE27DD6DCEF8
:2068C0008091C5078F5F863008F080E0A6CFEF92FF920F931F938C017B018091690490915C
:2068E0006A04B801A701F5D38091BE049091BF04B801A701EED31F910F91FF90EF9008952D
:206900000E949E230C943F274091E9064F5F4093E906642F70E09B012F5F3F4F8091C0076B
:2069200090E02817390724F04F5F4093C0074150E42FE150443190F09E2F0AC0292F2150E2
:20694000E92FF0E0E257F84F8081803219F4922F9923A1F79F5F9093E90610C0EE2319F1FF
:20696000E150AE2FB0E0A257B84F8C918032D9F411968C918032B9F4E093E906E091E906F8
:20698000E0938407F0E0E257F84F10821092E506B7DFF9DCAECC80E28083B9DD98DD8DE5C3
:2069A0008093C3040895FB01E257F84F8081882391F3F3CF0E940E240C943F278091C90737
:2069C000823011F4E0DCF6CF08956FEF40E050E043C3CF93DF931092580780910907A6DCB6
:2069E000982F80930907CEE5DDE101C02696FE0184919817D9F7F39B09C0F398CE010296E3
:206A0000FC0125913491F901099527C0F59B28C0F5982196FE01849189DCABDCFE013396FB
:206A2000C591D4912097C9F0D7FF06C09E012F77822F0E94BE2511C0CE01C7DF90936A043D
:206A40008093690480915807882339F0CE010496BCDF9093BF048093BE048EE10E94071388
:206A6000DF91CF9108958091760490917704892B19F086E794E081D380917B07833011F445
:206A800082E916C0843011F488EB12C010925B040E94F02280917B07853011F089EA08C07E
:206AA00080917C078350823010F08DEA01C084EB60DC8EE10E94071381E0809306030E9490
:206AC0006A280E940A1585DF8091290390912A03892B11F4ABDC57DC80910907883279F7B6
:206AE00080917B07833051F00E94B81784E18093A30781E080935B040E94F32280E00E94F0
:206B0000071381E08093540710920603D4C8CF93DF939091C3049E3539F48091C9078230F6
:206B200019F08FE421DC4FC0F39B17C0F398892F90E0805590409C01220F331F280F391F61
:206B4000220F331F2C5F324EF90185919491FC0109958EE10E94071336C0F59B34C0F598A5
:206B6000892F90E0805590409C01220F331F280F391F220F331F2A5F324EF90185919491D8
:206B8000FC0109952091C304822F90E080559040FC01EE0FFF1FE80FF91FEE0FFF1FE85F93
:206BA000F24EC591D491822F8F5F8093C3048F3508F08FE4D9DB209731F0CE0106DF9093CF
:206BC0007B0480937A04DF91CF910895FEDE90937B0480937A0408951F93182F8091760408
:206BE00090917704892B19F086E794E0C6D2112321F529DE80E5B8DB83E596E0E7DF8EE167
:206C00000E94071381E0809306030E946A280E940A157DDF8091290390912A03892B21F496
:206C2000CDDE8FE4A1DB04C08091C3048F3469F781E080935407109206031F9108958FEBBA
:206C400096E06FEF4AEE56E007D2909384048093830408959091C907923021F41092E906DE
:206C600036DCEDCF80918307981721F0892F0E949E273FCB08958CEF94E06FEF44EC56E072
:206C8000EBD190938404809383040895F4DFF59A08958091CD07C3D0882309F02ACB0895A9
:206CA0001F932BDB182F80917A07181749F087E090E0612F0E94D413812F0E94542319DB2E
:206CC0001F9108958091CC07882331F0F8940E946A1B0E942D150DCB08959091C7078091AB
:206CE0008607981721F0892F0E94AA2502CB08951F931091CB0780918707181749F0812FD8
:206D00000E94932384E190E0612F0E94D413F1DA1F9108959091C80780917E07981721F0CF
:206D2000892F0E94FA24E5CA08959091C60780910405981721F0892F0E94B827DACA08954D
:206D40009091C30780917907981721F0892F0E94F223CFCA08959091C2078091760798172B
:206D600021F0892F0E94DC24C4CA08959091C10780917707981721F0892F0E94FC23B9CA49
:206D800008959091C40780917C07981721F0892F0E94A727AECA08959091C50780917B0759
:206DA000981721F0892F0E94B425A3CA0895582F492F6F5F9C01F90106C08081882339F0D7
:206DC00031968C32D1F76150C1F75E2F4F2F852F942F0895DC018D91FB016F5F7F4FE491D6
:206DE0008E1711F080E008958C32A9F781E00895FC013181305180812AE0829FC001112442
:206E0000380F3C3308F031E0832F089580915707882321F00E940A151092570708958C331C
:206E2000A9F0982F995480918107882321F080918207981789F19093820781E08093810745
:206E4000809187078093750786E00AC080918107882311F1109282071092810780917507AC
:206E60000E9493238EE090E0609181070E94D4138FE090E0609182070E94D41384E190E023
:206E8000609187070E94D41382E090E0609175070E94D41381E0089580E008950F931F93D3
:206EA000CF93DF93082F162FC0E2D2E088EE94E0BE01F5D0892B89F4112321F0D093E904FA
:206EC000C093E80488EE94E0602F40E252E0C4D0FC01112311F017821682DF91CF911F912F
:206EE0000F910895EF92FF920F931F93DF93CF93CDB7DEB7CB54D0400FB6F894DEBF0FBE18
:206F0000CDBF109257077E010894E11CF11CC7016AE40E94EB148B3408F081C0C70166E7FC
:206F20007EE158DF882309F47AC0C70162E03FDFFC018081813409F072C01092540784E072
:206F40000E940713C70161E032DF8C0151DF8093D3060E5F1F4FC8014BDF8093D206C80130
:206F6000029646DF8093D106C70169E020DF8C013FDF8093D4060E5F1F4FC80139DF8093F3
:206F8000D506C801029634DF8093D606909182078091D306980F9093D30697FF08C0985E28
:206FA0009093D30681ED96E00E946A1609C0983138F098519093D30681ED96E00E94A016F4
:206FC0000E942C1E813011F40E94AF1681ED96E06CE674E046E050E0F1D2009781F0ACE66B
:206FE000B4E0E1EDF6E086E001900D928150E1F70E949E1C0E94BE1B81E080935307809164
:207000005307882329F00E947D1E84E160E006C080917607833019F084E061E03FDFC55B7D
:20702000DF4F0FB6F894DEBF0FBECDBFCF91DF911F910F91FF90EF900895809157078823F6
:2070400051F080915407882321F00E94EB22882309F0DCCE47CF0895DC01EAE0F7E030E089
:2070600080819181892B71F4B183A0838D919C91978386839383828381E0848365835187DC
:20708000408705C03F5F3A96363051F735E02AE0329F90011124265F384FC9010895AC0172
:2070A000EAE0F7E09F0180819181009741F08417950729F4808591858617970739F03A9611
:2070C00087E0E634F80771F720E030E0C90108950895FC01009749F0808191818617970799
:2070E00021F457834683538342830895DC01009771F0ED91FC91119716968D919C91179773
:20710000918380838AE0FD0111928A95E9F70895AAE0B7E021E08D919C911197892B39F1BE
:2071200015968C9115978F3F41F0815015968C931597882311F4CD01D9CF14968C911497FD
:20714000882329F018968D919C91199704C012968D919C911397ED91FC9111979183808397
:2071600014968C911497822714968C9314971A9687E0A634B80779F608950F931F938C01E3
:20718000FC0180819181B2DFF801118210821F910F9108951092B90081E18093B80008951E
:2071A000982F84EA8093BC008091BC0087FFFCCF8091B900887F883021F0803111F081E000
:2071C00008959093BB0084E88093BC008091BC0087FFFCCF9091B900987F983111F480E0BC
:2071E000089580E0903409F081E00895D9CF84E98093BC008091BC0084FDFCCF089580932A
:20720000BB0084E88093BC008091BC0087FFFCCF8091B90090E0887F883209F091E0892F3D
:20722000089584EC8093BC008091BC0087FFFCCF8091BB00089584E88093BC008091BC00E3
:2072400087FFFCCF8091BB000895A0E3B0E0EAE2F9E362C1A8E04E010894811C911CF401E4
:20726000BA2F1192BA95E9F729833A834B835C836D837E838F839887CE010996FC0111920D
:20728000AA95E9F7A986BA86CB86DC86ED86FE860F87188B29813A814B815C812DA73EA7B6
:2072A0004FA758AB79018A018FEF9FEFA0E0B0E0E822F9220A231B231A014424552429857A
:2072C0003A854B855C8529A73AA74BA75CA759016A01A822B922CA22DB223A0188249924A1
:2072E000C601B501A8019701A3D06DA37EA38FA398A7C401B3019CD069A37AA38BA39CA340
:20730000C601B501A201910193D07B018C01C401B3018ED05B016C0189A19AA1ABA1BCA1A1
:207320008E0D9F1DA01FB11F89A39AA3ABA3BCA32DA13EA14FA158A5CA01AA27BB2729A16F
:207340003AA14BA15CA1280F391F4A1F5B1F29A33AA34BA35CA32E153F054007510740F407
:2073600080E090E0A1E0B0E0A80EB91ECA1EDB1E89A19AA1ABA1BCA19D01442755272A0DF4
:207380003B1D4C1D5D1D2D8F3E8F4F8F58A36C01BB24AA248DA19EA1AFA1B8A5A070B070EC
:2073A000A80EB91ECA1EDB1EA98EBA8ECB8EDC8E9A8C8B8C7C8C9E8D6F8D78A1FE01719692
:2073C00088E0DF011D928A95E9F72D8B9E8B6F8B788F2D853E854F8558896DA57EA58FA542
:2073E00098A926D07B018C012D813E814F81588569A57AA58BA59CA51BD0E60EF71E081F7A
:20740000191F6D897E898F89988D6E0D7F1D801F911F6D8B7E8B8F8B988FEE892A2D392D1E
:20742000482D572D7E2F8F89988DE096E2E190C0629FD001739FF001829FE00DF11D649FEC
:20744000E00DF11D929FF00D839FF00D749FF00D659FF00D9927729FB00DE11DF91F639F2D
:20746000B00DE11DF91FBD01CF0111240895991B79E004C0991F961708F0961B881F7A9544
:20748000C9F780950895AA1BBB1B51E107C0AA1FBB1FA617B70710F0A61BB70B881F991FE6
:2074A0005A95A9F780959095BC01CD01089597FB092E07260AD077FD04D0E5DF06D0002009
:2074C0001AF4709561957F4F0895F6F7909581959F4F0895A1E21A2EAA1BBB1BFD010DC054
:2074E000AA1FBB1FEE1FFF1FA217B307E407F50720F0A21BB30BE40BF50B661F771F881F28
:20750000991F1A9469F760957095809590959B01AC01BD01CF0108952F923F924F925F9299
:207520006F927F928F929F92AF92BF92CF92DF92EF92FF920F931F93CF93DF93CDB7DEB730
:20754000CA1BDB0B0FB6F894DEBF0FBECDBF09942A88398848885F846E847D848C849B8434
:20756000AA84B984C884DF80EE80FD800C811B81AA81B981CE0FD11D0FB6F894DEBF0FBEF6
:20758000CDBFED010895FB01DC0102C005900D9241505040D8F70895FC010590061621F0B9
:2075A0000020D9F7C00108953197CF010895FB01DC0105900D920020E1F70895FB01DC01CD
:2075C00004C08D910190801921F441505040C8F7881B990B0895FA01CF93FF93EF93223003
:2075E000C4F02532B4F4C22F2C2F332744275527FF93EF936FDFEF91FF91605D6A330CF083
:20760000695D6193B901CA01605070408040904059F710828F919F91CF9114C0FB019F0139
:2076200042306CF045325CF4642F77272CDF805D8A330CF0895D8193CB010097A9F7108254
:20764000C90100C0DC01FC01672F71917723E1F7329704C07C916D9370836291AE17BF07B1
:08766000C8F30895F894FFCF70
:207B70000C94EC3D0C94FE3D0C94FE3D0C94FE3D0C94FE3D0C94FE3D0C94FE3D0C94FE3D2F
:207B90000C94FE3D0C94FE3D0C94FE3D0C94FE3D0C94FE3D0C94FE3D0C94FE3D0C94FE3DFD
:207BB0000C94FE3D0C94FE3D0C94FE3D0C94FE3D0C94FE3D0C94FE3D0C94FE3D0C94FE3DDD
:207BD0000C94FE3D0C94FE3D11241FBECFEFD8E0DEBFCDBF12E0A0E0B1E001C01D92A630E5
:207BF000B107E1F70E94A73E0C94F73F0C94B83D1124A5C00895982F8091C00085FFFCCFD5
:207C10009093C60008951F93982F82958F708A3018F0282F295A02C0282F205D892F8F7056
:207C30008A3018F0182F195A02C0182F105D822F0E94033E812F0E94033E1F910895982F07
:207C500007C08091C00087FFFCCF8091C60091509923B9F70895882309F483E090E0880F58
:207C700044EF51E00AC04E9A28EE33E0FA013197F1F721503040D1F79F5F9817A0F3089584
:207C9000CF93DF93C0E0D0E007C0219629F44E9A1D9902C00E94613F8091C00087FFF5CF58
:207CB0008091C600DF91CF9108951F930E94483E182F0E94033E113618F0812F875506C0CB
:207CD000103310F480E002C0812F80531F9108951F930E945D3E182F0E945D3E1295107FB2
:207CF000810F1F910895809104028F5F80930402853011F40E94613F08950E94483E803206
:207D100039F484E10E94033E80E10E94033E08950E947B3E08951F93182F0E94483E803232
:207D300051F484E10E94033E812F0E94033E80E10E94033E02C00E947B3E1F910895FF92D4
:207D50000F931F93CF93DF931092040284B714BE809160008861809360001092600080E403
:207D70008093C4001092C50088E18093C10086E08093C2005098589A569A2C9A2D9A1C9B2F
:207D900002C00E94613F88EA91E60197F1F71C9B02C00E94613F83E00E94333EFF240E9470
:207DB000483E803329F40E94853EFF24F394F7CFFF2021F488E080936000FFCF813341F4C2
:207DD0000E94483E803209F071C00E94EF3FE7CF803439F40E94483E8638E8F00E94483E42
:107DF0001AC0813499F40E94483E803811F482E020
:207E00005AC0813811F481E056C0823811F480E152C0883909F04EC083E04DC0823431F4CE
:207E200084E10E94273E0E94853EC1CF853411F485E0F7CF8035B9F38235A9F3813531F469
:207E40000E94853E88E080936000FFCF853549F40E94483E809300010E94483E80930101A4
:207E6000E2CF8635C9F40E94483E803389F40E94483E0E94483E182F0E94483E112311F489
:207E80008EE119C0113011F485E915C08FE013C083E00E94273E0EC0843621F40E94863F61
:207EA000000085CF843721F40E94C53F00007FCF863721F480E00E94933E79CF0E947B3E62
:207EC00076CF0C94000087B780FDFDCF07BFE89508951127103021F403E0F5DF01E1F3DF5E
:207EE0000990199001E0EFDF1395103428F0112705E0E9DF01E1E7DF3296129709F0EACFDD
:207F0000103011F01296F3CF11240895C1DEB82FBFDEA82FBDDE382FC2E0D1E0BD0177233D
:207F200009F0FFCF662321F0B3DE89936A95FACFAFDE803209F5E0910001F0910101EE0F3C
:207F4000FF1FC2E0D1E0353469F4AA2381F08991F999FECFF2BDE1BD80BDFA9AF99AAA9543
:207F60003196F3CFF999FECFA0FDA395B2DF84E14ADE80E148DE08958091040283958093C0
:207F8000040285300CF09DDF089582DEB82F80DEA82FE0910001F0910101EE0FFF1F78DE2F
:207FA000082F76DE8032A9F484E12DDE8A2F8B2B71F0053411F0859107C0F999FECFE1BD93
:207FC000F2BDF89A80B531961EDE1197EFCF80E11ADE08951441565220495350100008E00B
:127FE000E4EDFFE785910FDE0A95E1F70895F894FFCF67
:0400000500007B700C
:00000001FF
